:1000000000800020BD0100009D3C00009D3C0000E0
:100010009D3C00009D3C00009D3C0000693C0000B0
:10002000693C0000693C0000693C00009D3C000008
:100030009D3C0000693C00009D3C0000593C0000D4
:100040009D3C00009D3C00009D3C00009D3C00004C
:100050009D3C00009D3C00009D3C00009D3C00003C
:100060009D3C00009D3C00009D3C00009D3C00002C
:100070009D3C00009D3C00009D3C00009D3C00001C
:100080009D3C00009D3C00009D3C00009D3C00000C
:100090009D3C00009D3C00009D3C00009D3C0000FC
:1000A000A51D00009D3C00009D3C00009D3C000003
:1000B0009D3C00009D3C00009D3C00009D3C0000DC
:1000C0009D3C00009D3C00009D3C00009D3C0000CC
:1000D0009D3C00009D3C00009D3C00009D3C0000BC
:1000E0009D3C00009D3C00009D3C00009D3C0000AC
:1000F0009D3C0000AD5700009D3C0000295C0000C5
:100100009D3C0000D95F00009D3C00009D3C00002C
:100110009D3C00009D3C00009D3C00009D3C00007B
:100120009D3C00009D3C00009D3C00009D3C00006B
:100130009D3C00009D3C00009D3C00009D3C00005B
:100140009D3C00009D3C00009D3C00009D3C00004B
:100150009D3C00009D3C00009D3C00009D3C00003B
:100160009D3C0000994300009D3C00009D3C000028
:100170009D3C00009D3C00009D3C00009D3C00001B
:100180009D3C00009D3C00009D3C00009D3C00000B
:100190009D3C00009D3C00009D3C00001D3E000079
:1001A0006D3E0000F53E0000B13F0000354000000C
:1001B0009D3C00009D3C0000214F0000544B4CF240
:1001C000205210B51A804DF628121A8000BF00BFC9
:1001D00003F068FD4F4B4FF010621A604E4A9A6070
:1001E0004E4ADA604E4B1A6812F4807204D14D49BF
:1001F0000A604FF4A8521A604B4B1A7802F00802BA
:10020000D2B21AB11A7842F008021A70474B484825
:10021000484C2A221A700023474A02E01959995083
:10022000043399188142F9D3444B454A002101E037
:1002300043F8041B9342FBD34249434800231A5816
:100240005A500433B3F5DE7FF9D1404B404A802148
:1002500003F8011B9342FBD13A4A3E4B1A603E4BD6
:100260000A221A703D4B24221A70A02203F8012C96
:100270003B4A137803F00203DBB2002BF9D0384A73
:10028000137803F01003DBB2002BF9D1344A137852
:1002900003F00C03082BFAD1324B03221A704022D0
:1002A0005A702F4A137803F02003DBB2002BF9D0E9
:1002B0002B4A137803F04003DBB2002BF9D02A4B12
:1002C0002A4A1A6002225A60294B20221A70244AB4
:1002D000137803F00C030C2BFAD1264A264B1A6034
:1002E000264B274A1A60072243F8042C62B603F013
:1002F00045FF0C4B1B68DC0702D5224803F0B2FE19
:1003000007F0D8FF03F0D4FC04F0B6FEFEE700BF10
:100310000E20054030800440823F04000100002B85
:1003200010D0034014D0034002D0074000E0074043
:100330002895FF1F4CA30000608FFF1F2895FF1F0B
:10034000BC460020008AFF1F0000000000E400E01F
:100350005FE400E008ED00E0005006400140064088
:10036000064006400440064044800440000003016B
:1003700000400640C01005000480044014E000E086
:10038000FF76010023C97154FFFFFFFFFFFFFFFF4E
:10039000FFFFFFFFFFFFFFFFFFFFFFFFFFFFFFFF6D
:1003A000FFFFFFFFFFFFFFFFFFFFFFFFFFFFFFFF5D
:1003B000FFFFFFFFFFFFFFFFFFFFFFFFFFFFFFFF4D
:1003C000FFFFFFFFFFFFFFFFFFFFFFFFFFFFFFFF3D
:1003D000FFFFFFFFFFFFFFFFFFFFFFFFFFFFFFFF2D
:1003E000FFFFFFFFFFFFFFFFFFFFFFFFFFFFFFFF1D
:1003F000FFFFFFFFFFFFFFFFFFFFFFFFFFFFFFFF0D
:10040000FFFFFFFFFFFFFFFFFFFFFFFFFEFFFFFFFD
:1004100008B549F22850074BC1F6FF701B1A062B8E
:1004200000D808BD40F20003C0F20003002BF8D052
:100430009847F6E72B95FF1F08B549F2285049F277
:100440002853C1F6FF70C1F6FF731B1A9B1003EB14
:10045000D373591000D108BD40F20002C0F200026F
:10046000002AF8D09047F6E710B549F22854C1F6B3
:10047000FF74237873B9FFF7CBFF40F20003C0F29B
:1004800000032BB14AF24C30C0F20000AFF3008001
:100490000123237010BD00BF08B540F20003C0F275
:1004A00000034BB14AF24C3049F22C51C0F200002B
:1004B000C1F6FF71AFF3008049F22850C1F6FF701A
:1004C00003682BB140F20003C0F2000303B1984768
:1004D000BDE80840FFF7B0BF38B5054CA4F5964518
:1004E0002046103C04F07AFEAC42F9D138BD00BF82
:1004F000343F002038B5054CA4F596452046103C05
:1005000004F06CFEAC42F9D138BD00BF80E0FF1FA3
:10051000044A10B5044640F81C2B01F0DBFD2046D0
:1005200010BD00BF709D000038B5044608460D465A
:1005300003F0E8FB236802465B682046294698479B
:1005400038BD08B5FFF7F0FF08BD04F015BE0A225C
:10055000002304F0D9BD38B50446FFF7E5FF054692
:10056000204604F0C3FD281838BD38B5044604F011
:1005700003FE0546204604F0B9FD281838BDFFFFEC
:10058000044B00681B6882B00193019B181A02B0EB
:10059000704700BF94430020044B82B01B68019356
:1005A000019B591A016002B0704700BF94430020BC
:1005B0000F4B41720360002302610372C36019464E
:1005C00003E0026942F823100133427A9342F8DBD8
:1005D000084A136813B9106004E013465A69002AE8
:1005E000FBD15861002343618380C380704700BF03
:1005F000709900008C4400202DE9F0479CB08046A3
:1006000089460DF149070CA84146012201F042FF3D
:100610000CA801F0A4FD002800F0A0800CA801F0B7
:100620005FFD0146684604F01AFE68464E4904F034
:100630009AFE00283CD04D4908A804F010FE6846F8
:1006400008A904F087FE044608A804F0C7FD7CBB97
:100650004748484D04F0B5FE474B1A689042C8BF62
:1006600018604B260446464355F82000434B30188B
:1006700003EB001A0CA801F033FD0146504604F0CC
:1006800009FE55F824A00CA801F046FDB2443C4BED
:10069000374943F82A0055F824003A4B301803EB49
:1006A000001004F0EFFD55F82430013345F82430F4
:1006B0000CA801F017FD002846D0334904A804F027
:1006C000CEFD684604A904F045FE78B908A82F4974
:1006D00004F0C5FD684608A904F03CFED0F1010411
:1006E00008A838BF002404F079FD00E0002404A825
:1006F00004F074FD44B30CA801F0F2FC01461C4860
:1007000004F0C8FD9DF834308DF854300E9B1693DC
:100710009DF83C308DF85C301D4B0DF13D0214937B
:100720000DF15D0352F8041BBA4243F8041BF9D1E2
:100730003A781A70139B14A809F101011B93FFF773
:100740005BFF14A801F0C6FC0CA801F0FCFC684695
:1007500004F044FD0CA801F0BDFC54E70CA801F026
:10076000B9FC1CB0BDE8F087E4E0FF1F78990000F9
:10077000BC3F0020F4F3FF1F4495FF1F9095FF1F1F
:1007800004E1FF1F44F4FF1F7A99000080990000E4
:10079000689E000030B504468BB00A220D4601A8C1
:1007A000214604F087FD01A80B4904F0AEFD4B2360
:1007B0000A4903FB045401EB041101A804F0A0FD55
:1007C00001A805A91122002304F0E3FD01A804F00B
:1007D00005FD05A80BB030BD869900009095FF1F60
:1007E00008B54FF4FA7003F0B3FC024A024B1A60EA
:1007F00008BD00BF0400FA050CED00E010B504468A
:10080000C4F3C001062003F03DFC0520C4F38001C1
:1008100003F038FC0420C4F3400103F033FC032050
:1008200004F00101BDE8104003F02CBCFFFFFFFF06
:1008300008B572B6224A137F0BB10021117762B658
:10084000002B35D000211F48FFF7A6FE72B61C4BC7
:10085000B3F91E20B3F92000801A47F6FF72DA833D
:100860004FF400421A8462B607F04EF812A3D3E99F
:10087000002307F0D9F907F06FFB07F057F80022C3
:10088000114B07F0A7F807F03FFB07F03DF80246D1
:100890000B4600204FF0804105F082FD00220B4BFB
:1008A00006F0E4FE07F030FBBDE80840FFF7A6BF06
:1008B00008BD00BFAFF3008000000000E0FFEF4084
:1008C000483F0020A03F0020000014400000F03FFF
:1008D00010B5204B90B04FF080421A600446684635
:1008E00001F0EAFB1C491D4801F0CAFD1B491A4AE8
:1008F000132308A801F068FD9DF824308DF804301A
:100900000A9B02939DF82C308DF80C300DF12D03CD
:100910000DF10D0203F10C0153F8040B8B4242F868
:10092000040BF9D11B7813700F9B08A8079301F0F3
:10093000D1FB21466846FFF708FE684601F003FC3C
:10094000074B4FF080421A60684601F0C3FB10B0BD
:1009500010BD00BF88E100E08899000094400020AD
:1009600008E100E010B5244B244825494FF08044AD
:1009700090B01C6001F07AFD002837D0684601F085
:100980009BFB1E491E4A012308A801F01DFD9DF88E
:1009900024308DF804300A9B02939DF82C308DF89A
:1009A0000C300DF12D030DF10D0203F10C0153F884
:1009B000040B8B4242F8040BF9D11B7813700F9B88
:1009C00008A8079301F086FB684601F02EFBA0F112
:1009D0003004684601F029FB303802D40A2303FBB7
:1009E0000404684601F076FB204603E0FFF770FF41
:1009F000044B1C6010B010BD88E100E09440002062
:100A00008899000008E100E0F0B5904B1A7887B0B3
:100A10001C4632B18E4B1B781BB18E488E49FFF7B6
:100A200090FD23784BB18A4B1B7833B1172003F02C
:100A300029F801468748FFF788FD844B1A781C4641
:100A400032B1834B1B781BB182488449FFF779FD93
:100A500023784BB17E4B1B7833B1142003F012F88E
:100A600001467C48FFF771FD172003F00BF80446A0
:100A7000142003F007F8754B1A7824181D4632B17C
:100A8000734B1B781BB173487549FFF75AFD2B78E0
:100A900033B16F4B1B781BB16E482146FFF755FDF4
:100AA00040F2FF339C42A8BF1C46684B1A7824EAE8
:100AB000E4741D4632B1664B1B781BB16548694929
:100AC000FFF73FFD2B7833B1614B1B781BB16148B9
:100AD0002146FFF73AFD644B1A68644B53F8223005
:100AE0000021009320464FF480620B4604F06CFB1B
:100AF000564B1A7804461D4632B1554B1B781BB134
:100B000054485B49FFF71DFD2B7853B1504B1B78C0
:100B10003BB1554B4F481A68544B53F82210FFF71E
:100B200014FD4A4B1A781D4632B1494B1B781BB154
:100B300048485049FFF705FD2B7833B1444B1B78EB
:100B40001BB144482146FFF710FD4B4A4B4913683F
:100B5000086803934A4B039E1D6884420AD0701BA9
:100B6000052807D912680C6004924649049A0120AE
:100B700008701A6005250024152002F083FF064640
:100B8000162002F07FFF013D30440444F4D13A4A7C
:100B90003D4E1268052394FBF3F4022394FBF3F417
:100BA0000592374A059811683268640040F2FF33B5
:100BB0009C42A8BF1C4624EAE474A21A002AB8BFCB
:100BC0005242032A1ADD421A052A17D9264A116809
:100BD0002A4A12684B2000FB01212C4A2C4852F86B
:100BE0002150B5FBF3F303FB04F701F02BF8294A7E
:100BF0003460B0FBF5F005FB00751560264800F089
:100C0000E9FC20B1244800F0C7FC244B18702448AC
:100C100000F0E0FC20B1224800F0BEFC1F4B187031
:100C20002048FFF7ADFC0446082003F04BFA04FB14
:100C300000F11C48FFF7B0FC1A48FFF7A1FCB0F523
:100C4000C87F54D9084B18491A682FE0CCF3FF1F0E
:100C5000DCE0FF1FBC4400208C9900009D9900003F
:100C6000AE990000BD990000D8E0FF1FF4F3FF1F0C
:100C7000CB990000D899000094430020B43F002095
:100C80006C3F0020648FFF1FC4F3FF1F04E1FF1FB0
:100C90004895FF1FACE0FF1FF4E0FF1FCC3F002092
:100CA000D0F3FF1FD03F00204495FF1F0968013299
:100CB0008A421A6001DD00221A601F4B1F48012280
:100CC00000211A70FFF768FC00211D48FFF764FC43
:100CD0001C4B19781C4621B91B4B1C481A7800F094
:100CE00040FC23781BB1184B1868FFF7F1FD18483A
:100CF00000F070FCE8B1164800F04EFC012818D155
:100D0000114B1A6801320F2AC8BF00221A600A4B21
:100D100001221A700B4B19781C4621B90A4B0B485B
:100D20001A7800F01EFC23781BB1074B1868FFF7F8
:100D3000CFFD07B0F0BD00BF648FFF1FD03F002084
:100D4000E0F3FF1FDEE0FF1FD8E0FF1FD43F0020CD
:100D5000E4F3FF1F854B93F8443010B573B9844A10
:100D60001360844B01221A70834B1B7833B1834B81
:100D70001B781BB182488349FFF7EDFB7B4B1B7E41
:100D80005BB17D4B1B7833B17C4B1B781BB17C482E
:100D90007D49FFF7D6FBFFF723FD7C4B1B7823B97A
:100DA000744B1B78002B00F08880734B1B78002B52
:100DB00036D0724B1B78002B32D06C4C7449704883
:100DC000FFF7BFFB204600F03DFF01466C48FFF7F0
:100DD000BEFB70496A48FFF7B4FB654B6848196869
:100DE000FFF7B5FB6C496648FFF7ABFB614B644806
:100DF00019780A22002304F087F968496048FFF750
:100E0000A0FB624B5E4819780A22002304F07CF9AB
:100E100063495B48FFF795FB5948217EFFF7A5FB27
:100E2000604B1B783BB160486049002200F070FCC9
:100E30000F2003F08DF95E4B4D4C18685D4B19681F
:100E4000FFF7A8FC5C4B18604A4B1B781BB947485E
:100E500000F0F8FE2060584B22681968434822F0E1
:100E60000F02226000F08EFE0A2003F071F9424B5F
:100E70001B7873B1414B1B785BB150494048FFF779
:100E800060FB3B4B3E481968FFF761FB3C4804F0B0
:100E90002DF9444B1B7823B143484449012200F00B
:100EA00037FC434B1868FFF7A9FC384B4448002136
:100EB0001970304B1970FFF76FFB4248FFF760FB6A
:100EC000414B1B68984205D9FFF79EFD3D48002124
:100ED000FFF762FB284C23784BB33C48FFF750FBED
:100EE0003B4B1B68984238D821E0244B1B781BB140
:100EF00023483849FFF725FB1F4B1A781C464AB197
:100F00001E4B1B7833B1194800F09CFE01461C486B
:100F1000FFF71DFB237833B1184B1B781BB1184822
:100F20002D49FFF70EFB29480021FFF735FB244828
:100F3000FFF726FB09288CBF002101210B2003F0BD
:100F4000A1F82648FFF71CFB29280ED92448FFF7F3
:100F500017FBB0F5FA6F04D810BD2378002BC4D16D
:100F6000CAE7BDE81040FFF763BC10BD4895FF1FFE
:100F7000ACE0FF1FCC3F0020CCF3FF1FCDF3FF1FE1
:100F8000BC440020E1990000EE990000648FFF1F2F
:100F9000FF9900001A9A0000269A00002F9A00007C
:100FA0003A9A0000CEF3FF1FB0E0FF1F3AFF620045
:100FB000D8E0FF1FB43F0020443F0020439A0000C8
:100FC000E0E0FF1FB83F0020688FFF1FC8F3FF1F3E
:100FD0006C8FFF1F529A0000699A0000A03F00200A
:100FE000E0F3FF1F2DE9F84F2B4EDFF8D080DFF83C
:100FF000D090002429492A48FFF7A3FA214628481F
:10100000FFF7B3FA56F8041F2548FFF79EFA254963
:101010002348FFF796FA2449214804F046F84FF494
:10102000967A1F4821494FF04B0BFFF794FA0AFBC1
:10103000048A00250BFB04FB26E0294605EB0B0781
:101040001748FFF782FA3F0119491548FFF779FA67
:1010500009EB0701124804F028F816491048FFF779
:1010600070FA15490E48C91904F01FF811490C48C7
:10107000FFF767FA5AF825100948FFF768FA084899
:101080000C49FFF768FA013533689D42D5DB01341E
:10109000102CAFD1BDE8F88FF0F3FF1F8D9A000040
:1010A000BC440020A29A0000E4E0FF1F949A0000D4
:1010B000A19A0000A49A00009095FF1F04E1FF1F71
:1010C00044F4FF1F30B5022089B0002103F006F878
:1010D0000820002103F002F80920002102F0FEFFA1
:1010E0000B20012102F0FAFF0620012102F0F6FF99
:1010F0000520012102F0F2FF0420012102F0EEFFA1
:101100000320012102F0EAFF734B1868FFF776FB1A
:10111000724B1A781C461AB14FF47A7003F018F823
:10112000237833B16E4B1B781BB16E486E49FFF7C5
:1011300012FA6E48052103F0EDFD684B1B7833B1C0
:10114000674B1B781BB167486949FFF704FA694B85
:101150001A7842F005021A70604B1B7833B1604B6D
:101160001B781BB15F486449FFF7F5F963480A2112
:1011700001F08EF8C0B1594B1B78F3B924E0237805
:101180002BB12B781BB157485D49FFF7E4F90F20CD
:10119000FFF734FB642002F0DBFF0020FFF72EFB9B
:1011A000642002F0D5FF01E04C4C4D4D53480A211C
:1011B00001F06EF80028E2D0DDE7494B1B781BB147
:1011C00048485049FFF7C7F94C494F4A0123684640
:1011D00001F0FAF84D4A9DF804301371029B9360B8
:1011E0009DF80C3013730DF10D030D3203F10C015A
:1011F00053F8040B8B4242F8040BF9D11B78434C93
:101200001370079B6846E36100F064FF334B1B7863
:1012100033B1334B1B781BB132483D49FFF79BF983
:1012200023798DF80430A3680293237B8DF80C306A
:10123000384B0093384B0DF10D0203F10C0153F8BC
:10124000040B8B4242F8040BF9D11B7813702F4B1F
:10125000DB69684600210793FFF7CEF9684600F086
:1012600039FF1E4B1A781C4632B11D4B1B781BB13F
:101270001C482A49FFF76FF9237823B1184B1B78D4
:101280000BB1FFF7AFFE264B19781C4619B925485C
:1012900000F064F900E0002023781BB1FFF762FB47
:1012A000002809DB204B1B68984205DC0A4B1860BC
:1012B0001E4B01221A700CE0194B19781C4619B903
:1012C00018480A4600F04DF9237813B10020FFF7C3
:1012D000FFFA09B030BD00BFD8E0FF1FCCF3FF1FFD
:1012E000DDE0FF1FBC440020A89A00000082FF1F21
:1012F000B79A0000B6440020C59A00009440002030
:10130000D99A0000F69A000086990000803F0020DC
:10131000089B0000689E00008D3F0020169B000087
:10132000DEE0FF1FD43F00204495FF1F648FFF1FA6
:101330002DE9F041674D684F684EDFF81C820021AF
:1013400086B00A462846FFF733F9654B2846002445
:1013500040F81C3B00F0B0FE284600F0EFFB2846AA
:101360006049614A06F088FF012107F124023846EE
:10137000FFF71EF95D4B06F118023B6030464FF057
:10138000FF330121BB61FFF713F9594B336047F677
:10139000FF7308F118020121F38340464FF4004324
:1013A0003384FFF705F9534B4046C8F8003000F08E
:1013B0007BFA514880E8A00004724472C46003F0D4
:1013C00082FD4E4880E8800104724472C46003F0DC
:1013D0007AFD4B4880E8600004724472C460494D55
:1013E00003F071FD4849494803F039FF474848492F
:1013F0003D4A06F041FF05F596460AE020460021E9
:10140000103403F02CFFAC42F8D104F59665B542D8
:1014100002D0A5F59664F1E73E4D3F49324A0020DF
:1014200006F02AFF05F596460AE020460021103412
:1014300003F015FFAC42F8D104F59665B54202D031
:10144000A5F59664F1E7284A3449002006F014FF18
:101450003349344803F003FF2D49234A314806F04D
:101460000BFF314800F028FE30491F4A2E4806F095
:1014700003FF082114222E4800F07AF809210A22DD
:101480002C4800F075F8022114222B4800F070F867
:101490002A4B1A6800920099294A11601A68019231
:1014A0000199284A11601A6802920299264A11602D
:1014B0001A6803920399254A11601A6804920499E4
:1014C0001B68234A05931160224B059A1A6006B0E7
:1014D000BDE8F0814895FF1FB0E0FF1F483F0020A6
:1014E000709D000011050000608FFF1F509D0000DF
:1014F000409D0000609D0000703F0020A43F002040
:1015000034F4FF1F409AFF1F2B9B0000E4E0FF1FF5
:10151000DD510000F4F8FF1FF5040000D9040000BD
:101520002F9B0000BC3F0020803F0020D520000002
:10153000F4E0FF1FD0F3FF1FE4F3FF1F94430020EC
:10154000C8F3FF1FE0E0FF1FD03F0020B83F00209E
:10155000E0F3FF1FA03F002090E0FF1F084602F0CD
:101560004DBB0846114602F05DBB02F00BBBFFFF0E
:1015700037B500238360074B42601B680193019BD2
:101580000446036008460D4602F09CFD6573207317
:1015900020463EBD94430020007B704713B50446AF
:1015A000407B02F08FFD237B834201D100200EE0BF
:1015B000074B1A68009200992268891A6268914262
:1015C000F4D31B6820730193019B012023601CBD91
:1015D0009443002037B50446FFF7E0FF10B1002325
:1015E000A3600EE0A26872B1084B19680091009DDB
:1015F0002168691A914206D31B68A0600193019B80
:101600002360012000E00020A0733EBD9443002031
:1016100070B50021044603F028FCC0B1B4F91E20C7
:10162000B4F92030811C00F5817631F9025BAA42C1
:10163000A8BF2A46AB42B8BF2B46B142F5D323849C
:101640000123E2832377BDE8704003F0D9BB70BD6E
:101650002DE9F047846905462CB9214603F005FCC5
:10166000002851D04CE00021631C0BD103F0FDFB9E
:101670000446002848D028462146002203F0E0FB1B
:1016800020463DE003F0FEFB064600283CD0EA6918
:1016900095F820101D4800234FEA146CC4F30F2E58
:1016A00030F91CA00CF1010CF71830F91CC0B7F987
:1016B0000280CEF580390EFB0CFC0AFB09CE4FEA06
:1016C0002E4E0EFB08FE4FEAEE3EA7F802E021B1D7
:1016D000E743BA4205D2A41807E0A24204D2A41AF2
:1016E00003E04FF0FF3400E00C460233B3F5807F97
:1016F000D2D12846AC613146002203F0A1FB30462E
:10170000BDE8F04703F07CBBBDE8F087329B0000EA
:1017100072B683690BB9012303E0013302D16FF084
:1017200001038361C16180F8202062B67047FFFF2A
:101730002DE9F041DFF860C0154E164F002A0CBFAE
:101740004FF064524FF06052002434F8078056F88E
:1017500014509CFBF8F8414504D303F00801C9B2CA
:1017600021B905E002342E2CEFD1F6E742F0806279
:1017700003F00403DBB23BB125F4704305F470457C
:1017800042F0007243EA15152A430260BDE8F08179
:10179000009E0000D09D0000006CDC0210B50446E5
:1017A000FFF7C6FF204610BD10B5044603F04AFC03
:1017B000204610BD02480349034A06F05DBD00BF44
:1017C000D83F0020A9170000608FFF1F024803497F
:1017D000034A06F051BD00BFE03F0020A9170000FA
:1017E000608FFF1F10B5194B1A6811681A79184BD2
:1017F0001A70184A9142184928BF184B08683CBF14
:10180000134603F5807298B1014631F9024F04F591
:10181000FF447F34241123F8024B9342F5D303F0A5
:10182000EFFA0F4B0C491A680A6000221A6005E0B3
:1018300040F2FF7123F8021B9342FBD3094B1B7844
:101840001BB1094B4FF080421A6010BDEC3F0020E5
:101850001F8000400A88FF1FF83F00200A87FF1FF3
:10186000E83F0020F43F002008E200E010B500212E
:1018700003F0FBFA034690B172B60949086808B94B
:101880000B6003E0074A146814B9136062B610BD18
:101890000C60136062B6BDE8104003F0B1BA10BD31
:1018A000F83F0020E83F002038B54B484B4D012160
:1018B00003F070FB4A4B1A6842F480521A60494B9D
:1018C00080221A7000242C8008340120A4B202F077
:1018D0003FFCB4F5006FF6D1434B1B685B0264D547
:1018E000424B1A6848F6A273134048F6A27293421C
:1018F0005BD13F4B1A6840F23F439A4255D13D4B72
:101900001B68012B51D13C4B1A6840F201139A42DB
:101910004BD1314D39492B681A6819600221197170
:1019200019726FF0010159734FF0FF319973D97338
:1019300019692A494FF4807019610022D98AD88226
:1019400011465A715A729A72DA721A731A755A7566
:101950001A765A769A76DA76DA8BD8839A8B0124BD
:1019600006229A839C71DC712B7903F1804303F585
:101970000433B02219701A7003F0BCFA204B214ACC
:1019800018702B792048137003F110011F4A42F898
:1019900021005A11920002F1604202F5614203F007
:1019A0001F0304FA03F4146038BD0F4B1A6842F4A5
:1019B00080021A600F4B01221A6040F23F4243F846
:1019C000082C48F6A37243F80C2C114A43F80C2C4F
:1019D00040F201125A609CE7EC3F002000C00C402E
:1019E0002C80044021C00C403C8004400060034037
:1019F000046003400C600340106003400A87FF1F2F
:101A0000F43F00201B800040E5170000008AFF1F04
:101A1000A28F010002480349034A06F02DBC00BF13
:101A2000EC3F0020A9170000608FFF1F0248034908
:101A3000034A06F021BC00BFFC3F0020A9170000AC
:101A4000608FFF1F02480349034A06F015BC00BF20
:101A500004400020A9170000608FFF1FF8B590F820
:101A600044300446002B61D003F082F9054600287B
:101A70005CD004F11C06304600F052FB00283BD03D
:101A8000A91C30464FF4807200F034FBB0F5807F23
:101A900007461ED926492748FEF746FD0A2200239D
:101AA0003946244803F030FB224803F01FFB304640
:101AB00000F049FB204A1388002B2FD0013B9BB23A
:101AC0001380002B2AD0002384F84430012323768E
:101AD000F8BD236CC318236400232376470803E072
:101AE00005EB470201375380802FF9D12046294664
:101AF000002203F0A5F90CE0304600F024FB0E4A6A
:101B000013887BB1013B9BB213805BB1002384F847
:101B100044302846BDE8F84003F072B95E2000F07A
:101B200035FAD0E75E2000F031FAEFE7F8BD00BFEC
:101B3000789D0000BC4400200C400020002380F869
:101B40004430C3630364704708B572B690F84430FC
:101B500073B1002380F8443062B61C3000F0F3FA11
:101B6000074A138833B1013B9BB2138013B108BD00
:101B700062B608BD5E20BDE8084000F007BA00BFAD
:101B80000C400020F0B589B0154604460F46FFF71B
:101B9000DBFF5E2000F0E0F9254B1A8801321A8045
:101BA00072B624493A460123684600F00DFC9DF8C0
:101BB000043084F82030029B63629DF80C3084F876
:101BC00028300DF10D0304F11C0604F1290203F184
:101BD0000C0153F8040B8B4242F8040BF9D11B782B
:101BE0001370079B6846A36300F074FA62B6304630
:101BF00000F0B5FA074628B90F481049FEF7ABFCCC
:101C0000384613E0304600F087FA0346B5FBF0F1A2
:101C100003FB1151E063304600F072FA2564064878
:101C20000749FEF798FC012084F8440009B0F0BD94
:101C30000C40002094400020BC4400207C9D00000B
:101C4000949D0000006C7047094B1B7813B9094B39
:101C50001B782BB1084A1378202B03D90123037179
:101C6000002070470548C1540133137001207047AC
:101C700072400020354000207340002014400020B6
:101C80007047FFFF024B1878024B1B78C01A704751
:101C90007140002070400020064A074913780978F7
:101CA000994204D90549C85C0133137070474FF05D
:101CB000FF30704770400020714000203640002007
:101CC000054B064A1B7812789A4202D9044AD05C26
:101CD00070474FF0FF307047704000207140002087
:101CE0003640002038B50E4B1B78144613B90D4B07
:101CF0001B788BB10C4B1D78C5F121039C4202D996
:101D0000012202711C4609482246401906F00CFEC9
:101D1000054B2D191D7000E01C46204638BD00BF44
:101D20007240002035400020734000201440002005
:101D300010B5104B1B7813F020040BD1122002F0C9
:101D400055F80D4B1B68A3B10C4A14700C4A10785F
:101D5000984710BD0B4A13780133DBB2012B137087
:101D600002D8094B1B7823B91220BDE8104002F0BD
:101D70003DB810BD036006401040002070400020B8
:101D8000714000205C40002035400020002202719C
:101D90000273034A4FF47A7181600260704700BF9A
:101DA000B89D000010B5374A137803F01001C9B28E
:101DB00021B903F04002D2B242B92EE010211170D5
:101DC00003F04002D2B2002AF3D110BD13F0040395
:101DD0002D4A18D0002313702C4A13702C4B1B680B
:101DE000144603B1984722782A4B1AB927491A702A
:101DF00001200870284AD02111701A78274B1A70D8
:101E00000122274B21E001211170264A1370224B39
:101E1000C0221A7002331B7830E01F4A1F4C117821
:101E200011F0100117D013F0010310D11C4917480D
:101E30000A780078904205D9164B9B5C01322370DA
:101E40000A7000E02370144BD0221A7016E0C023F1
:101E50001370237812E0144B1220197003221349D7
:101E600001F09AFF0F4A207813781F2B06D80649F5
:101E7000097819B10E49C85401331370014B02227D
:101E80001A7010BD036006400E4000207340002011
:101E900058400020144000200260064004600640C4
:101EA00074400020714000205C400020311D000083
:101EB000364000200148FFF769BF00BF60400020A6
:101EC000184B19491A6842F480521A60174B184A85
:101ED0001A60184A116001F180415160164A1A6077
:101EE000164B1B78DA0755BF154A164A4FF4107186
:101EF0004FF40071116003F00201C9B24FF4007297
:101F000009B9114900E0114903F00403DBB20A608A
:101F10001BB94FF410720E4B02E00E4B4FF40072DF
:101F20001A6070473C8004400110003800C0024035
:101F300001401F000CC0024000001F80B64400207A
:101F400018B0044008C004401CB004400CC0044059
:101F500014B0044004C004405E2830B511D8094ACA
:101F600043091478012101FA03F52C431470064A41
:101F700000F01F0052F8234001FA00F10C4342F830
:101F8000234030BD90400020784000205E2810B5EE
:101F900014D843090A4A00F01F0052F823400121D7
:101FA00001FA00F024EA000042F8230030B9054AA3
:101FB000107801FA03F320EA0303137010BD00BF89
:101FC000784000209040002013B502AB026803F86F
:101FD000011D546819460122A0471CBDC06908B103
:101FE00001F01CB8704738B50446C069002510B927
:101FF0000123237138BD0571E06992B201F090F9B7
:10200000E3691B7913B101232371284638BD07B555
:1020100001220DF1070100F0F1FE01280CBF9DF82F
:1020200007004FF6FF7000B20EBDC06908B510B1D1
:10203000FFF7EDFF08BD4FF0FF3008BD38B505468E
:10204000C06950B1FFF7E3FF431C044606D0E869BE
:10205000C168013900F0AEFF00E00446204638BDFB
:10206000F8B504464FF47A73A360124B0020207138
:102070002073236024200D46174606F047F9E061DF
:10208000A8B12B4603F120020546186859682E4670
:1020900003C6083393423546F7D118683946306095
:1020A0000C2204F10D0007F0EFF9002363762046BF
:1020B000F8BD00BF689E00004FF47A71816004494A
:1020C0000022027102730160C2614273704700BF57
:1020D000689E0000014B0360704700BF689E0000CF
:1020E0000D307047C06920B18079012894BF00206D
:1020F00001207047C06908B508B100F07FFE08BD37
:10210000C06908B100F056BF7047C3690BB1D86809
:1021100070474FF0FF307047C06900B18069704769
:1021200038B5C369044663B1FFF7F6FF054620469C
:10213000FFF7EBFF47F6FF73281A984228BF1846AF
:1021400038BD184638BD10B50446C06930B100F03E
:1021500091FFE06906F0E2F80023E36110BDC06979
:1021600018B18079003018BF0120704710B50A46B9
:102170008AB00A49044600238DF8083001918DF891
:102180000A30214601A8012301F02AF8044610B1C3
:1021900001A800F06FFF20460AB010BD989E000015
:1021A0000AB101F0A5B80120704770B50B68C45C96
:1021B0002F2C08BF0133C6180024355D2F2D08D001
:1021C0006DB906E001330B60C05C003018BF012020
:1021D00070BD00251555C25C2F2AF4D1F2E71555C4
:1021E000013401330C2CF4D0E7E7FFFF2DE9F04F69
:1021F0009A4699B0254B00248DF81C408DF81E405E
:102200008DF840408DF84240019480460D4691463D
:1022100006930F930C4606AE04E0234600E00FAB96
:1022200034461E4601A902AA4046FFF7BEFF80F0D1
:102230000102074602A92046D2B25346C847834648
:1022400038B9AC4201D100201DE0204600F012FF59
:10225000F9E777B101233046214602AA00F0C0FF1A
:10226000AC4207460CD0204600F004FF002FD4D12A
:10227000E9E7AC4202D0204600F0FCFE012002E07B
:102280000028CCD1DFE719B0BDE8F08F989E0000A0
:1022900038B590F83E3004460D4613B1383000F0A2
:1022A000E9FE204601212A4600F0D0FA08B90020B4
:1022B00038BD04F1100501222846214601F094FAA8
:1022C000024640B104F13800294600F06FFD0030AD
:1022D00018BF012038BD2846214601F085FA0028A4
:1022E000E5D0EFE70A7902710A4A02604A79427141
:1022F0008A7982718A688260CA68C2600A690261EA
:102300000A7D02758A698261CA69C2610A6A0262CB
:10231000704700BF989E00002DE9F04F97B005462A
:10232000383104A891469A46FFF7DCFF254B4FF061
:10233000000B8DF838B00D938DF83AB04C460DAFC8
:1023400004AE2DE023782F2B01D1013428E0C4EB1B
:1023500000085FFA88F8B8F10C0F28BF4FF00C089E
:1023600021464246684607F08FF816AA02EB08039A
:10237000384603F858BC00F07DFE384631466A46C0
:10238000012300F02DFF20B90E4B28712B60A8719E
:1023900014E0304600F06EFE334644443E461F468D
:1023A00020462F2106F04EFE0028CBD1C9EB0404B5
:1023B000CAF8004028463146FFF794FF284617B078
:1023C000BDE8F08F989E0000F0B59DB004461E4613
:1023D00001A86B461746FFF79FFF009BFD18FB5CAB
:1023E0003BB901A913A8FFF77DFF204613A91C4A9A
:1023F00030E000238DF82C301A4A8DF82E309DF8ED
:102400000A300A921BB92046FFF756FE24E0023B31
:10241000012B0AA806D814492A46334600F0E0FEEC
:1024200050B9F0E701A92A46334600F0D9FE00284A
:10243000E9D001A800F01EFE16F0060F03D00AA88E
:10244000109900F0B7FD0AA913A8FFF74BFF20462B
:1024500013A92A46FFF704FE20461DB0F0BD00BFB9
:1024600086990000989E0000CC40002000F13803BF
:10247000024A084619460023FFF7B8BE6D21000046
:1024800000F13803024A084619460023FFF7AEBEA2
:10249000A121000070B504469EB00D46164628E006
:1024A0009DF8100000B92AE0E52822D02E2820D07F
:1024B0009DF81B0000F00800C0B2D0B9134B8DF896
:1024C00034008DF83600694604A80C9300F01EFC19
:1024D0000CA8E9696A46334600F082FE78B10CA97F
:1024E00015A8FFF7FFFE204615A96A46FFF7B8FDBD
:1024F00008E0E86904A900F015FD0028D0DC2046BA
:10250000FFF7DAFD20461EB070BD00BF989E0000A8
:10251000084B02211961084900225A719A719A7276
:102520001A7383F8302083F83C20996383F83E20A7
:10253000704700BF94400020989E0000094B1A6825
:1025400042F480621A602C334FF000421A60064A4F
:10255000FF2111601A68002AFCDA044B1868C0B227
:10256000704700BF00C0024034C0024038C0024083
:102570001A4B1B4A70B51A60C307044602D5FFF711
:10258000DDFF013C052C01D8630800E00323002295
:102590001449154801E0086001329A42FBDB23EA46
:1025A000E372A4EB42040F49104A0F48104D06E0B5
:1025B000166816F0F00FFBD008602E68023C002C65
:1025C000F6D106E0106810F0F00FFBD00868013B70
:1025D00001E0064A0649002BF4D170BD00C002405C
:1025E00000041F8034C00240FFFF00902CC0024056
:1025F00038C00240074B1A6842F480621A602C33DC
:102600004FF000421A60044A10601A68002AFCDA8F
:10261000704700BF00C0024034C0024013B5114CE7
:10262000052813D8DFE800F0030306090C0F01A802
:102630000D490DE001A80D490AE001A80C4907E089
:1026400001A80C4904E001A80B4901E00B4901A8CD
:1026500000230122FFF7A2F8019B2360FFF730FC63
:102660001CBD00BFF440002000366E0100127A004D
:1026700000093D00C0C62D0080841E00801A06009F
:1026800010B5194B1B780BB3DA0707D5174A184951
:10269000146809682140174C2160116003F00202A0
:1026A000D2B23AB1144A1249146849682140114C17
:1026B0006160116003F00403DBB23BB10F4B0C4AC5
:1026C000196892680A400B498A601A600C4A1368BC
:1026D000834208D00B4B0C491960106040F08040D9
:1026E00050600A4A1A6010BD9040002080E100E06E
:1026F000784000208440002084E100E088E100E090
:102700000CC0024000C0024001401F0000001F80BA
:102710000C4B1B78ABB1D90703D50B4A11680B4A98
:10272000116003F00202D2B21AB1074A5168084A96
:10273000116003F00403DBB21BB1034B9A68054B35
:102740001A607047904000208440002000E100E0C3
:1027500004E100E008E100E008B50121007901F0A2
:1027600091FCFFF7D5FF08BD054B10B5044618686E
:10277000FFF786FF20790021BDE8104001F082BC00
:10278000F440002010B5837904468BB1008940F2F3
:102790000123984207D8C0F500700230FFF7E8FE29
:1027A00040F2022323812046FFF7D6FF0023A371C6
:1027B00010BDFFFF73B50B4B1A680092009E0D46CB
:1027C0001C46B6B2FFF7BAFEFF2808D02368019373
:1027D000019B9BB29B1BAB42F4DB002000E001207D
:1027E0007CBD00BF94430020F8B505460E46174651
:1027F000FFF7C8FF2846FFF7B7FF4FF4967128464A
:10280000FFF7D8FF46F04000FFF7F4FE182427FA40
:1028100004F0C0B2083CFFF7EDFE14F1080FF6D14A
:1028200026B1082E0CBF8720FF2000E09520FFF77F
:10283000E1FE0024FFF782FE0306E87204D5FF2CB8
:1028400002D00134E4B2F5E7F8BDFFFF2DE9F04313
:1028500000230373837283714371544B027185B0FB
:102860001B680446019310460F460121019E01F0AA
:1028700035FC0121207901F005FC4D4B1A6842F42A
:1028800080521A600620FFF7C9FE4A4B1868FFF70E
:10289000F7FE0A25FF20013DFFF7ACFE15F0FF050E
:1028A000F8D1FFF735FF2046FFF75EFFDFF8FC8029
:1028B0001FFA86F90BE0D8F800300293029B9BB216
:1028C000C9EB0303B3F5FA6F01DD01234EE00021EC
:1028D00020460A46FFF788FF01280546E072EAD144
:1028E000204608214FF4D572FFF77EFF00F0040068
:1028F000C0B208B125730DE00425FFF71FFE013DAE
:1029000015F0FF05E072F8D1AA284FF0020300D0BD
:102910002CE02373257BDFF89480022D0CBF4FF051
:1029200080450025B6B20AE0D8F800300393039B37
:102930009BB29B1BB3F5FA6F01DD082316E037212C
:1029400000222046FFF750FF2A4620462921FFF7A4
:102950004BFF0246E0720028E6D1237B022B15D103
:1029600020463A21FFF740FF10B10623637115E0BE
:10297000FFF7E4FD00F0C000C02801D1032323735A
:10298000FFF7DCFDFFF7DAFDFFF7D8FD2046FFF784
:10299000E3FE3846FFF742FE012003E02046FFF742
:1029A000DBFE002005B0BDE8F08300BF94430020AB
:1029B0003C800440F440002073B5114B1A6800922B
:1029C000009E04461D46B6B209E02B680193019BA8
:1029D0009BB29B1BB3F5967F01DD0F2307E0FFF74A
:1029E000ADFDFF28E072F0D0FE2806D00D23204672
:1029F0006371FFF7B1FE002000E001207CBD00BF45
:102A0000944300202DE9F843089D04460F46904664
:102A10001E4603B974E09B18B3F5007F73DC83791D
:102A20002BB10368994202D10389934216D9237BC3
:102A30002760032B18BF7F023A4620461121FFF77B
:102A4000D3FE074610B1032363715CE02046FFF715
:102A5000B3FF002857D001232781A3714046FFF719
:102A600087FD2C492C4B1960F107324604D5FFF73E
:102A700065FD05F8010B721E052A01D8530800E018
:102A8000032300212548264F01E0076001319942C8
:102A9000FBDBA2EB4302AA182248204FDFF880C0DC
:102AA000DFF884800DE0016811F0F00FFBD0C7F86B
:102AB00000C0D8F80010C1F3072985F800906970AC
:102AC00002359542EFD302EB43031748154A09E05C
:102AD000116811F0F00FFBD00168C1F307272F70C8
:102AE000697002359D42F3D32389F618A37AB6B2F2
:102AF000268113B1B6F5007F02D32046FFF742FED0
:102B00000120BDE8F8832046FFF726FE0020BDE83F
:102B1000F88300BF00041F8000C0024034C00240A0
:102B2000FFFF00902CC0024038C0024007B54FF4B0
:102B3000007300920022FFF765FF0EBD2DE9F04102
:102B400004462B482B4F03682B4D43F480634FF012
:102B5000004603603E6029603946002307468C46E4
:102B6000D1F800E0BEF1000FFADA12E0D1F800E08F
:102B7000BEF1000FFADA18E01E4A1368002BFCDAE7
:102B800026E0112320466371FFF7E6FD0020BDE833
:102B9000F081D0F8008012F803E048F48068C0F8B3
:102BA00000800E60C5F800E0E0E702EB030ED7F806
:102BB00000809EF801E0023348F48068B3F5007F9E
:102BC000C7F80080CCF80060C5F800E0C8D1D3E7B2
:102BD000FF20FFF70FFDFF20FFF70CFDFFF7AEFC16
:102BE000E07200F01F000528CBD10120BDE8F08184
:102BF00000C002402CC0024034C0024070B50B46F9
:102C00000446164609B9122329E0027B032A18BF9D
:102C10004B021A461821FFF7E7FD054608B10423C9
:102C20001DE02046FE213246FFF788FF88B120468E
:102C30004FF41671FFF7BEFD08B915230FE02046CB
:102C40000D212A46FFF7D0FD40B9FFF777FC28B9E0
:102C500007E02046FFF780FD002070BD142363715C
:102C6000F7E72046FFF778FD012070BD014A024BCF
:102C70001A60704701100138F440002010B5044676
:102C80000121006A04F1080200F032FD40B1E3695D
:102C90002BB9A368E361637963F07F03637101205B
:102CA00010BD70B50446FFF7E9FF08B9002070BDFC
:102CB000236AA268197C1D79023A02FA01F65A6960
:102CC000B218561E06E0701900F056FC0028EDD030
:102CD000013DEDB2002DF6D1236A1B7C4FF400724A
:102CE00002FA03F2A3699B18A361012070BDFFFFE4
:102CF00010B50446006900F01BFC18B1207D024BA2
:102D000003EB401010BD00BF04410020002230B58D
:102D100013462E24855C202D09D0D5B2082D02D172
:102D2000CC540133DBB2855CCD540133DBB20132CC
:102D30000B2AEFD10022CA5430BDFFFF70B500232B
:102D400005462022CA5401330B2BFBD10022072455
:102D50001FE02E2B01D0144E06E00A2C22D00822B0
:102D60000A2416E098421DD016F8010F0028F9D168
:102D7000A24218D8202B16D97E2B14D8A3F16106B5
:102D8000192E01EB020001D8203BDBB201320370A7
:102D9000D2B215F8013B002BDBD10878203818BFE0
:102DA000012070BD002070BD7F9E000038B5827983
:102DB00004460D460AB1002038BD91F82030102B92
:102DC00006D1022383714B8CC2615B0183610CE0ED
:102DD000202BF0D103238371496A04F11802C161E9
:102DE000284600F019FC0028E5D0002301202562C8
:102DF0006071A360E3602361237538BD2DE9F04F56
:102E0000837985B00446904613B94FF6FF7865E0A4
:102E10004379DB07F9D564E01FFA83F847460E468D
:102E2000DFF8F890DFF8F8A056E0E268A179206AB0
:102E3000D3054FEAD35B02291FFA8BF34FEA522ED8
:102E400002D1416A71441CE00579013D05EA0E0595
:102E5000EDB26BB965B912B9E269A26008E0A16888
:102E6000039304F1080200F0A3FB039B0028CCD0DD
:102E7000226AA168107C5269023901FA00F18918AE
:102E80004919CBF500729742627902F04002C8BF3F
:102E9000C3F50075D2B2CCBFADB23D4612B9B5F59F
:102EA000007F2ED1DAF80020914220D129E0761956
:102EB0000DE00BEB090358191A46314603E012F8EE
:102EC00001CB01F801CB8242F9D1D31AF618E3689D
:102ED0007F1B5B19E360BFB2002FA6D10FFA88F009
:102EE00016E08269C368D31A984595D896E70A4ACE
:102EF000009610681A462B46FFF784FD0028D6D1AD
:102F000083E70846002100F013FB0028D1D17CE7BD
:102F100005B0BDE8F08F00BF004100200441002053
:102F2000708FFF1F38B58379012B05460C4601D8F9
:102F3000FF201BE0C368DA06FAD10AE02278A2B1CA
:102F4000E52A06D02E2A04D0E27A02F00802D2B294
:102F500062B1202228462146FFF750FF42B2202AC4
:102F6000ECD0002AE4DB002000E0104640B238BD7F
:102F700037B58379012B044601D8002016E0C368D9
:102F800001220DF10701C3F34315FFF737FF0128B5
:102F90000CBF9DF807304FF6FF731BB20133ECD026
:102FA000E26803481F32E26000EB45103EBD00BFFF
:102FB00004410020F8B5044680790D4600282CD045
:102FC000A369994224D825E01DB9A560E5600120D8
:102FD000F8BD236AE2681E7C691E0936531E23FA77
:102FE00006F321FA06F69E4200D312B9E369A36004
:102FF00009E0F61A07E0206AA1683A4600F0D8FA1C
:10300000013E10B9F8BD04F10807002EF3D1DDE749
:103010000020F8BD0228D7D1D8E7F8BD38B58379AC
:10302000054613B390F90530002B1ADA0121FFF79A
:103030005FFE0446C8B1AB79012B9CBFAB69C3618D
:10304000EB6943831B0C8382094B1B682BB118303F
:1030500004F116019847238B63826B7903F07F0399
:103060006B71BDE8384000F03DBA002038BD00BFAC
:10307000F840002010B50446FFF7D0FF10B1002340
:10308000A371012010BDFFFFF7B58279012A044624
:103090000D4645D1437903F00203DBB2002B3FD04C
:1030A00040E0002B3AD0E668FFF784FF00B937E034
:1030B000206A35B9E16900F073FB002830D0E56182
:1030C0001BE0A16801AA00F073FA48B3206A184B0C
:1030D00090F8207001994FF6F872102F08BF134630
:1030E00099420AD200F05CFBD0B1206AA1686FF06F
:1030F000704200F0B9FA00B912E06379A56163F09B
:103100007F0363712046FFF789FF48B12046B5422F
:1031100034BF29463146FFF74DFF07E0104605E072
:10312000002003E083699942BBD9F9E7FEBD00BFE7
:10313000F8FFFF0F10B500210446FFF7A5FF60B1AF
:1031400020460121FFF7D4FD38B1E52303700023A9
:10315000A371BDE8104000F0C5B9002010BDFFFF0D
:1031600038B51D4B03EB41131546DA7A12F0110FF7
:10317000044604D015F0420F01D0002038BD174A94
:103180002175126822615A8B998A42EA0141E161F4
:10319000DA7A12F0180203D1DB69A361012309E096
:1031A000102AEAD1206A04F1180200F035FA00284A
:1031B000E3D00423A37105F00F0305F040050021BF
:1031C000EDB26371A160E16025B12046BDE83840F1
:1031D000FFF75ABF012038BD04410020708FFF1F48
:1031E0002DE9FF47867905460C461F46002E75D10E
:1031F0000DF1040810464146FFF7A0FD00B96DE04F
:10320000236AA6602B62E660DFF8E090C24621E008
:103210002046C3F34318FFF7ABFE014600285DD0FC
:1032200002780AB1E52A09D126B9D9F8002085F833
:1032300014802A610B78012683B10BE050460B22E3
:1032400005F040FB30B907F03003302B46D028465C
:1032500041463FE0E368A2699342D9D307F01203E5
:10326000122B3BD136B128460121FFF741FD044620
:1032700048B933E0A379022B30D02046FFF711FD87
:1032800060B3184C2E7500212022204601AE05F0B7
:103290006BFC03CE20606160B3783288A372124B5E
:1032A00022811B682BB104F1100004F10E01984734
:1032B00006E021222274A373282208236274E37398
:1032C000238A63822383E389E38200F00BF928B128
:1032D000297D28463A46FFF743FF00E0002004B06E
:1032E000BDE8F08704410020F8400020708FFF1FE8
:1032F00010B50A468AB00949002304468DF8083003
:1033000001918DF80A3001A821460223FFF768FFDA
:1033100010B101A8FFF70EFF0AB010BD989E000083
:103320002DE9F74F92468279012A07460C4640F074
:10333000B680427902F00201C9B2002900F0AF80E4
:10334000B1E0B969FD688D4201D1554688E0FFF7CB
:1033500031FE002800F0A380F7E7386A90F804B047
:103360000BF1FF3B0BEA522B4FEAC2594FEAD959F6
:103370001BF0FF0B1FFA89F81FD1B8F1000F1CD109
:10338000B96811B9FA69BAB911E001AA00F010F9E7
:10339000002800F08F80396A474891F82010019A80
:1033A0004FF6F873102908BF1846824204D33846F6
:1033B000FFF764FC08B972E0BA603A6AB968107C39
:1033C0005269C8F500760239B6B2B54238BF2E460A
:1033D00001FA00F18918B6F5007F8B4411D1374A04
:1033E0001168594504BF4FF0FF311160344A594606
:1033F00010682246FFF702FC002850D004F5007444
:1034000029E0B8F1000F10D1F968BA6991420CD3E4
:1034100000F068F8002842D0284AC2F800B0294AD3
:10342000117841F00101117005E05846012100F0CA
:103430007FF8002833D0244A914409EB0600611E2E
:103440004A4603E011F801CF02F801CB8242F9D1DC
:10345000C9EB02094C44FA68AD1B9619ADB2FE6087
:10346000FA68002D7FF479AFB9698A4201D9BA614F
:1034700005E0164A126832B1BAF1000F03D07A792A
:1034800062F07F027A717A7902F00802D2B20AB948
:1034900050460FE03846FFF7C1FD0028F8D1012261
:1034A0003A71002006E002F00402D2B2002A7FF452
:1034B00048AF4AE7BDE8FE8FF8FFFF0F708FFF1F90
:1034C000004100200443002004410020F840002077
:1034D00007B502AB012203F8011D1946FFF720FFD3
:1034E0000EBDFFFF38B50D4B1B78A3B10C4D0D4B36
:1034F000286819680C4AFFF781FB68B10B4C2168FA
:1035000031B12868084AFFF779FB28B1002323600E
:10351000024B00221A70012038BD00BF0443002076
:1035200000410020708FFF1F04410020FC4000205C
:1035300070B50D4D2B68834204460E460DD0FFF743
:10354000D1FF08B9002070BD084B094A1868214610
:10355000FFF7ECFA0028F5D02C60064B1A781643DA
:103560001E70012070BD00BF708FFF1F0041002042
:10357000044100200443002010B50446FFF7B2FFC9
:1035800078B10023074A194699540133B3F5007FF7
:10359000FAD1054B1C60054B1A7842F001021A70F3
:1035A000012010BD04410020708FFF1F0443002044
:1035B000C3680133994270B505460C46164601D9D9
:1035C000002070BD95F82030C069102B01D10B0A86
:1035D00000E0CB0918180E4B1B68984205D195F8EE
:1035E0002030102B0B4B0AD105E00021FFF7A0FF84
:1035F0000028F4D1E4E7E4B233F8143005E004F035
:103600007F0453F8243023F070433360012070BDF1
:10361000708FFF1F044100202DE9F74302AEDFF851
:10362000448046F8041D0546174600244FF6F879F5
:10363000284601993246FFF7BBFF80B12B7C4FF43F
:10364000007202FA03F395F82020E418019B102A77
:1036500014BF42464A469342EAD33C600120BDE88B
:10366000FE8300BFF8FFFF0F0129F8B504460D46A1
:10367000174633D9C368013399422FD890F82030C8
:10368000C669102B01D10B0A00E0CB099E19144B1F
:103690001B689E4205D194F82030102B114B0BD1A2
:1036A00006E030460021FFF743FF0028F3D1F8BDC4
:1036B000EDB223F8157003E005F07F0543F825709F
:1036C000094B1A7842F001021A70237E012B03D9AC
:1036D000A368F618054B1E600120F8BD0020F8BD58
:1036E000708FFF1F0441002004430020FC40002095
:1036F0002DE9F74F156806468A4617461DB1013574
:103700004FF0000905E04B1ED3F10009056859EBA5
:103710000309F3682C4603F1010B4FF00008F3682E
:1037200098451CD25C4501D90224254630462146E5
:1037300001AAFFF73DFF90B1019A631C0AB11D4633
:1037400002E05B1B534503D008F101080134E6E7B2
:10375000304621466FF07042FFF786FF58B90020CF
:103760001CE004F1FF38304641462246FFF77CFF5B
:103770000028F4D04446AC42F3D8396821B93D6002
:10378000B9F1000F07D108E030462A46FFF76CFF79
:103790000028F4D1E3E7013535600120BDE8FE8F54
:1037A000F7B502230F4F036005460C464FF6F87637
:1037B0002846214601AAFFF7FBFE80B12846214694
:1037C0000022FFF751FF50B195F82030019C102BDB
:1037D00014BF3B4633469C42EAD3012000E0002060
:1037E000FEBD00BFF8FFFF0FF8B53B4B0446196064
:1037F0001546CAB1042A01D90020F8BD00200146AF
:10380000FFF796FE0028F7D0344B03EB051505F5BE
:10381000D475AA795206EFD1D5F81220632AEBD9D4
:10382000D5F80E50002DE7D028460021FFF780FE86
:103830000028E1D0294BB3F80B20B2F5007FDBD193
:103840001A7C002AD8D0D9890029D5D05B7B002BDF
:10385000D2D02276002223712274012003E0511C71
:10386000072A2174C8D8227C00FA02F18B42F6D1D3
:103870001A4BD98A01B9596ADE89A160AE19E6618D
:10388000B3F811001F7C6084400107FB016100F266
:10389000FF10616201EB50216161B3F813300BB985
:1038A0000E4B1B6A691ACB1823FA02F240F6F47326
:1038B0009A42E26001D80C2309E04FF6F4739A4271
:1038C00001D8102303E0054BDB6A6362202384F8F0
:1038D00020300120F8BD00BF00410020044100203D
:1038E000F0B53048304903681B06FCD40B6813F070
:1038F0008002F8D172B62D4B1978002950D02C498E
:1039000008684F688E68CD680C69381814318019C2
:103910000968401900194018C0F34E00254940F4C9
:1039200000400860C86A0F6B4E6B8D6BCC6B38180B
:10393000403180190968401900194018C0F34E0041
:103940001D4940F40040086001F10811143151F89C
:10395000140C51F8107C51F80C6C51F8085C51F8BB
:10396000044C096838188019401900194018C0F330
:103970004E00124940F400400860C86A0F6B4E6B5D
:103980008D6BCC6B381840318019096840190019CB
:103990004018C0F34E000A4940F4004008601A7015
:1039A00062B6F0BD24B0034024B00B4006430020B3
:1039B00038B003402CB0034030B003402CB00B4073
:1039C00030B00B40224B60221A70E1225A70214B1A
:1039D000214A1978214B082901D1012102E00A2945
:1039E00007D13921116013221A601D4B19605A60EA
:1039F0000BE00C291A4901D1352000E03D20106070
:103A000012221A60174B08601A60174B17491B786F
:103A1000174A03B101230B601360164B164A19783D
:103A2000164B012901D880210CE0042901D88421FA
:103A300008E0082901D8852104E0102901D8862151
:103A400000E08721116019600D4B01221A70704748
:103A500000400740748FFF1F08B003400CB00340C4
:103A600008B00B400CB00B400943002020B00340CD
:103A700020B00B40758FFF1F24B0034024B00B40D3
:103A8000064300200D282DE9F0410FD9172801D851
:103A90000E380AE0A0F11A03052B01D8093804E01A
:103AA000A0F12203062B4DD81838C0B2274B1C5C5E
:103AB000274B1B780BB1FFF713FF72B6200614D407
:103AC000244D254E01272C60377062B672B62B68E4
:103AD000190603D5214B18681F4B23E03378002BC0
:103AE000F1D062B601F072FCF0E704F040071C4D23
:103AF0001C4EFFB204F03F044FF001081A4B1A6845
:103B000017B122F0100201E042F010021A602C609E
:103B100086F8008062B672B62B681A060BD5134B76
:103B20001868104B00221A7062B6114B1B7840FACD
:103B300003F0BDE8F0813378002BDFD062B601F0EE
:103B400045FCE8E70020BDE8F08100BFA09E000032
:103B50000643002000B003400843002010B003409B
:103B600000B00B40074300200CB00B4010B00B40DE
:103B700005430020024A1378DB07FCD5704700BFDD
:103B80000100024030B5194B85B06C4603F11005B9
:103B900018685968224603C20833AB421446F7D16D
:103BA000134B1B7803F00203DBB2BBB1114B802235
:103BB0001A7033221A710322DA7072B60E4C6B46F9
:103BC00043F001032046984762B6237813F0700350
:103BD00004D0237008E0013B03D105E0044944F61A
:103BE00021630A78D207F6D505B030BDB89E000033
:103BF000010002400700024000000240B0F5006FE3
:103C000010B5044609D2064B1B78D90701D4FFF73B
:103C1000B9FF04F1A054207810BD002010BD00BFF2
:103C200001000240B0F5006F38B504460D460FD2D2
:103C3000084B1B78D90701D4FFF7A4FF04F1A05467
:103C40002378AB4204D02570BDE83840FFF792BF1F
:103C500038BD00BF01000240024B1A6801321A60F1
:103C6000704700BF9443002038B50B4C25462368AD
:103C7000580301D500F090FB2B68590501D501F0E0
:103C800095FD2B681A0501D501F0CEFF2368DB04F2
:103C9000EDD502F0A1F9EAE73480044008B5FFF75A
:103CA000E3FFFFFF014B10221A8070470020054000
:103CB0007047FFFF024A13681818106018467047D3
:103CC000788FFF1FFEE7FFFFEFF313839BB9EFF33E
:103CD000108098B9EFF3058323B10F2B04D9084A5C
:103CE000985C01E04FF48070EFF311833BB1984290
:103CF00028BF184670474FF0FF307047184670478E
:103D0000F0E300E0002300E00133C25C002AFBD1B5
:103D10001846704710B50023B0FBF2F402FB140004
:103D2000092801D8303000E03730C85420460CB1A3
:103D30000133F1E7CA185470224605E0885CCC5C78
:103D40008C54C8540132013B9A42F7DB084610BD3F
:103D5000031E10B50C4603DBBDE81040FFF7DABFC9
:103D60002D2001F8010B5842FFF7D4FF204610BD6B
:103D7000084B4FF400021A604FF080721A604FF047
:103D800000721A604FF080621A604FF000621A6091
:103D9000704700BF08E100E0212830B521D8042A8F
:103DA0001FD8DFE802F00709050B03000B2306E02C
:103DB0000A2304E0082302E00C2300E00923094A57
:103DC00002EBC002526872B61468074D24F47024E6
:103DD000146044F0807444EA034345F820101360F3
:103DE00062B630BDC89E00000C430020094B03EBB7
:103DF000C0035B6872B61A6822F0877222F48032C0
:103E000042F080721A60044B002243F8202062B610
:103E1000704700BFC89E00000C430020114B10B536
:103E20001C68E0041C6004D50F4BDA680AB1DB683B
:103E30009847A10404D50C4B1A690AB11B6998472D
:103E4000A20604D5084B1A6E0AB11B6E9847E3060A
:103E500006D5054BD3F8842012B1D3F884309847A7
:103E600010BD00BFA09004400C4300201F4B10B5B4
:103E70001C68E0031C6004D51D4B1A680AB11B685E
:103E80009847A10304D51A4B5A680AB15B68984752
:103E9000E20704D5164B1A6C0AB11B6C9847A307AE
:103EA00004D5134B5A6C0AB15B6C9847200704D5B4
:103EB0000F4B9A6C0AB19B6C9847610704D50C4B69
:103EC000DA6C0AB1DB6C9847220304D5084B5A6EB2
:103ED0000AB15B6E9847630306D5054BD3F8802083
:103EE00012B1D3F88030984710BD00BFA0A00440A5
:103EF0000C4300202C4B10B51C6820071C6004D517
:103F00002A4B5A6A0AB15B6A9847E10604D5274BE7
:103F10009A6A0AB19B6A9847620604D5234BDA6A0B
:103F20000AB1DB6A9847230604D5204B1A6B0AB105
:103F30001B6B9847A00604D51C4B5A6B0AB15B6BF0
:103F40009847E10704D5194BDA6B0AB1DB6B984748
:103F5000A20704D5154B9A6D0AB19B6D984763076C
:103F600004D5124BDA6D0AB1DB6D9847A00504D574
:103F70000E4BDA6E0AB1DB6E9847E10504D50B4BA8
:103F80001A6F0AB11B6F9847620504D5074B5A6F29
:103F90000AB15B6F9847230504D5044B9A6F0AB1A9
:103FA0009B6F984710BD00BFA0B004400C43002099
:103FB0001E4B10B51C68E0071C6004D51C4B9A68AA
:103FC0000AB19B689847210604D5194B5A690AB172
:103FD0005B699847E20604D5154B9A690AB19B695B
:103FE0009847630704D5124BDA690AB1DB69984731
:103FF000200704D50E4B1A6A0AB11B6A9847A1071D
:1040000004D50B4B9A6B0AB19B6B9847A20604D55B
:10401000074B1A6D0AB11B6D9847630604D5044B14
:104020005A6D0AB15B6D984710BD00BFA0C0044037
:104030000C430020094B10B51C68A2071C6004D576
:10404000074B9A6E0AB19B6E9847E30704D5044B61
:10405000DA6F0AB1DB6F984710BD00BFA0D00440F3
:104060000C430020044B054900221A600A60044AF0
:10407000106010221A60704714D0034004D003402F
:1040800000D00340212810B518D80D4A52F830301E
:1040900093F880423CB1012211B183F8802010BD19
:1040A00083F8002110BD02EBC00043681A6811B10B
:1040B00042F0030201E022F002021A6010BD00BFCC
:1040C000C89E0000212805D8034B53F8303093F8E0
:1040D0000002704700207047C89E0000212816D8B3
:1040E0000B4A02EBC00301295B6852F8302004D16F
:1040F00082F880124FF4A27208E0002082F8800259
:1041000011B94FF4807201E040F203121A60704757
:10411000C89E000072B60B4B0B491A680B4B1B680C
:10412000096862B6490102D5322A88BF0133C2F557
:10413000BB32FF326021B2FBF1F24FF47A7000FB28
:104140000320704718E000E004ED00E094430020F5
:1041500070B50446FFF7DEFF05466CB140F2E73666
:10416000FFF7D8FF401BB04203D9013C04D005F54E
:104170007A7501F02BF9F3E770BDFFFF10B5FFF77B
:10418000F7FD164B164A174C00204BF6FF711860CE
:1041900059602823136093601361936113629362E3
:1041A00013639363092222600F4C20606160A36057
:1041B000236144F8042C0D4C20600D4801600D492A
:1041C0000B608B600C4B1A60FFF7FCFB0420FFF7C1
:1041D000BFFFBDE8104000F0FBBB00BF0480034000
:1041E0000C800340008003400490034004800B4097
:1041F00008800B400C800B4000800B40F0B50C4B4E
:104200000C4C1A7842F0020504EBC50682F001025C
:10421000706009481A700678002E0CBF8827C827DE
:1042200047EA014186F0010644F835100670F0BDFA
:10423000004400200080FF1F78440020431E032B11
:1042400010B510D872B6094A52F8230048B1416837
:1042500042F82310064A018832F81340611A22F806
:10426000131062B610BD002010BD00BFF043002047
:10427000A8460020013803280BD872B6064B53F825
:104280002030002001E05B680130002BFBD162B6DA
:1042900070470020704700BF4444002070B572B6DC
:1042A000184E194C01239A1912F8012C02F0080239
:1042B000D2B2E2B19900144A54F831502DB902EB50
:1042C000431308305860114B09E041F0010154F8E4
:1042D000315065B902EBC103083058600C4B42F80D
:1042E00031300C4B1A78013A1A7062B670BD013346
:1042F000052BD8D162B6074B00221A70BDE870407A
:1043000000F0D2BB00A000000080FF1F880040002A
:10431000C80040006E440020431E032B30B532D845
:104320004001194A40F01000101872B6174CE25CB8
:10433000032A09D8DFE802F0160218050830022225
:1043400013E00830042210E01148124A50F82340CC
:1043500014B940F8231002E052F82300416042F8FB
:1043600023100FE0032200E00522E25410F0080FB2
:1043700001F108030A8843600CBF8823C82343EA7D
:104380000243036062B630BD0080FF1FAC430020D3
:1043900044440020544400202DE9F74FA54EA64C7C
:1043A000357805F00403DBB2ABB1A44B1B7883B1C5
:1043B000A34A137823B1013BDBB2137003B900BEEB
:1043C000A04A13782BB1013BDBB213700BB900F09C
:1043D0007FFC0423337005F00802D2B2002A00F0FB
:1043E0008082994B1B781D094FEA930940F0FE81AA
:1043F00004EBC903586854F83930C3F38303013B15
:104400000C2B00F2F081DFE813F0A901A901EE0105
:10441000EE01EE01EE01EE01EE01C501EE01EE014D
:10442000EE010D004368894902684B60884B89485A
:1044300044F83930884D0A60002303600120287059
:1044400092B240F28165AA422361A36117D8B2F506
:10445000D06F80F02C81B2F5817F00F0DC8006D82F
:10446000802A00F0C280822A40F03D81C1E040F203
:1044700002339A4200F00C81B2F5A06F16E042F2CE
:104480002105AA4200F0678108D8B2F5086F00F054
:10449000A680B2F5106F40F026810AE042F221209A
:1044A000824200F01C8142F221339A4240F01B818B
:1044B0001DE18A78614B604D1A702B6A180603D58E
:1044C000686A083800F0F0FA644A08359542F4D179
:1044D000DFF8B091DFF8B0B10025A846CA4655F81C
:1044E000090005E04368009300F0DEFA009B1846DF
:1044F0000028F7D15A4B4AF8050045F80B00E85858
:1045000007E042680093019200F0CEFA019A009B06
:1045100010460028F5D15851524BE850524B23F821
:104520001800524B18F80320023A032A08D8DFE893
:1045300002F002040204002200E0012203F8082035
:1045400008F101080435B8F1040FC8D1484BDFF871
:104550003C9100221A7001259846464B05EB090252
:10456000EB1812F8012C9B001A7002F00802D2B26C
:104570003AB300F07BFAAB0038B104EB45120830D7
:1045800050603D4A44F8332006E044F8330098F880
:104590000030013388F8003000F068FAAB0043F0D7
:1045A000010338B104EBC30208305060284A44F8D4
:1045B000332006E044F8330098F80030013388F8DF
:1045C0000030AA0042F00201013542F0030200234C
:1045D000052D44F8313044F83230BED188E0174B15
:1045E000264D1B782B70034685E0244D2B706B7095
:1045F00080E08A88042A00D975E0204D2B706B700A
:104600001F4B9200D3181B7803F00203DBB2002B80
:1046100070D028706EE08A8802F07F03042B62DC81
:104620004B8803B15FE09100154A8A18117821F098
:10463000020156E0802007400080FF1F77440020E1
:104640000144002079440020902007406444002069
:10465000C800400098430020784400208080FF1F5D
:104660004444002054440020A8460020AC430020CD
:104670006E44002030C80110880040006F440020C4
:10468000C0200740F04300209C43002000A0000011
:104690008A8802F07F03042B25DC4B8803B122E0DB
:1046A0009100A14A8A18117841F0020119E04A8864
:1046B0009E4B898853F8085CA3F10C009DB133F838
:1046C0000CCC944509D133F80ACC8C4505D1120A9B
:1046D000032A0CBF2B7803890DE00C33EAE78978B5
:1046E000934A117004E0904B0F221A7033E00023BC
:1046F0001D4600E002238F4AB2F806904B4538BFB2
:104700009946B9F1400F34BFC8464FF040082846DB
:104710004146FFF773FDB9EB0809454403D1B8F1F1
:10472000400F07D017E0B9F1400F34BFC8464FF033
:10473000400800E0C84628464146FFF75FFDB9EB58
:104740000809454402D1B8F1400F04D17A4B7B4AA5
:104750001D60A2F800900122794B43E0754B1A8846
:1047600042F221039A4211D1764A0023C15C995446
:104770000133072BFAD1734B1B68862B02D1724B86
:104780000F221A7000200146FFF738FD6F4B44F8E6
:10479000393028E0684BD3F80080B8F1000F18D00A
:1047A000DFF89891B9F800A0BAF1400F34BF554630
:1047B000402540462946FFF721FDC5EB0A039BB281
:1047C000A9F800300BB9402D01D108EB05035A4A76
:1047D0001360584B1A88B2F5A06F04D100225A70AA
:1047E0009A785B4B1A700122554B6DE004EBC908B7
:1047F00003F00803D8F80420013DD9B2A2F1080063
:10480000EDB2002937D000F04FF95248524B50F822
:104810002510F1B14A6840F8252001F10802C8F8D6
:1048200004205A5D032A0BD8DFE802F002040608D0
:10483000032204E0022202E0052200E004225A558D
:1048400018F0080F0A880CBF8823C82343EA0243E4
:1048500042E05A5D032A07D8DFE802F04040020434
:10486000002206E0012204E018F0080F0CBF02222B
:1048700003225A5532E054F839301B0C22F8083C18
:1048800023B322F8061C42F8041C344A344952F877
:10489000257017B942F8250002E051F82520506034
:1048A000304A41F8250032F815105B1822F815300F
:1048B00000F0DCF818B10830C8F8040006E02A4B14
:1048C00044F839001A7801321A7007E01F4B274A62
:1048D00018F0080F08BF134644F839300823337026
:1048E0005EE5E90752D516492048214C02230B709A
:1048F000204B1A70204B1860986020481A61D860CD
:104900009A615C60084B0D2018701D48FF230370EE
:1049100000F8083C02741B4A13701B4B9F221A704C
:1049200001230B704BE000BFC020074010A0000027
:104930008844002064440020984300206C440020F8
:1049400094200740B046002001440020C8004000E9
:104950009820074044440020AC430020F04300204E
:104960009C430020A84600206E44002088004000A0
:10497000B0430020004400200080FF1F04440020BA
:10498000882007408C200740842007402B0605D54F
:104990000C4B0D221A70802203F8402C05F0020304
:1049A000DBB22BB1084B1A781A70022203F8082CDC
:1049B00005F01005EDB215B1044B10221A70BDE8D8
:1049C000FE8F00BFC020074088200740802007409E
:1049D00008B501F057FB00231E491A465A50C81863
:1049E0000833882B4260F9D11B4B1A6842F48022AD
:1049F0001A601A4B80221A701978184A0906FBD4DB
:104A0000144B1749C3F307200870C3F307401B0E6C
:104A100008750B76FF2301F81C3C01F8143C01F8E3
:104A20008C3C137843F0400313700021012302F8FB
:104A3000783C02F80C1C02F8883C0A4B70226FF498
:104A4000507C1A7063444FF400721A60064B1022B7
:104A50001A7008BD0080FF1F348004400C210740FD
:104A60009C20074049E400E00821074072B60C4A48
:104A70001168B1FA81F30B2B02D962B6002070479E
:104A80004FF0004020FA03F021EA0001116062B605
:104A9000044948225343C8180022CA504260704754
:104AA0007C8FFF1F008CFF1F0C4B4822C31AB3FBE7
:104AB000F2F30B2B11D80A4A127822B1094A127864
:104AC0000AB1FFF7EBBB72B6074A4FF0004121FA7B
:104AD00003F311681943116062B67047008CFF1F21
:104AE0006E440020774400207C8FFF1F38B5114CA6
:104AF00023684BB10F4D28684288811801320C7A27
:104B000001888A4212D30CE00B4B1B7813B94FF08B
:104B1000FF340CE00320FFF791FB20600028E9D16F
:104B2000F5E7FFF7C1FF00232B6000E0428020463D
:104B300038BD00BF844400207744002010B50C4CE1
:104B400023681BB10A4B1B686BB902E0094B1B7849
:104B500013B94FF0FF3010BD0320FFF76FFB20604B
:104B60000028EFD1F5E75A889B18187A10BD00BFCE
:104B70008444002077440020044B9888044B1B6831
:104B80001BB11A885B88D31AC0187047A84600204A
:104B9000844400202DE9F8432D4B2E4DDFF8C080D2
:104BA00001220C461A7006464BE02B682BBBDFF83F
:104BB000A0904AF2F92798F8003013B9244A1370EC
:104BC00014E00420FFF756FB072808D8012389F8D2
:104BD0000030FFF74BFF286078B989F80000013FEB
:104BE0001D4B01D01A782AB101221A704FF0FF3004
:104BF000BDE8F88300F0EAFBDDE72968164A48883B
:104C000000231370C0F14002944238BF224600F1E5
:104C100008078018CF194880A41A02E0F05CF85405
:104C200001339342FAD1F6184B883F2B06D9402323
:104C30000B800420FFF770FB00232B60074B05223D
:104C40001A70002CB1D1024B20461C70BDE8F883CD
:104C50007A4400207C4400208044002079440020D5
:104C60007744002007B502AB012103F8010D184677
:104C7000FFF790FF0EBDFFFFF8B5114B1B78EBB1AE
:104C8000104E114B3468114D01271F704CB16388D1
:104C900000272F70042023802146FFF73DFB37605B
:104CA00009E0FFF7E3FE014620B104202C70FFF776
:104CB00033FB00E02F70044B00221A70F8BD00BFD8
:104CC000774400207C4400207A440020794400206E
:104CD00038B50D4B1D78ADB90C4C216831B14B88FE
:104CE00004200B80FFF718FB256038BDFFF7BEFEE0
:104CF000014620B10420BDE83840FFF70DBB044B4E
:104D000001221A7038BD00BF7A4400207C44002084
:104D100079440020F0B5C02928BFC02172B6124BDB
:104D20001860124B00221A605A609A60DA601A61A9
:104D30005A6101260AE0540902F01F0753F8245073
:104D400006FA07F73D4343F8245001328A42F2D174
:104D500000234FF4817203E002FB0304637001330C
:104D60008B42F9D162B6F0BD944400209C440020EF
:104D700010B572B61E4B1868A0B9586850B998683B
:104D800050B9D86850B9186950B95869143348B93E
:104D900062B610BD043305E0083303E00C3301E0D4
:104DA0001033FFE7B0FA80F14FF0004222FA01F22F
:104DB00020EA020018600F4802780132D2B2027075
:104DC00062B60B481B1A9B105B01591A4FF4817392
:104DD0004B43094903F5F9531E3309680124CC54A8
:104DE000C818064B1978914238BF1A7010BD00BF21
:104DF0009C440020994400209444002090440020CA
:104E0000417872B60378012B02D9013B037011E09F
:104E10004A11094BC9434FF0004001F01F0120FA2D
:104E200001F153F82200084343F82200034B1A789B
:104E3000013A1A7062B670479C44002099440020E1
:104E400030B5C3680EE0187A90420AD158685C7A8F
:104E5000006950F8245025B940F824100878013032
:104E60000870DB68002BEED130BD437A99424FF0D9
:104E7000000305D2026952F8210042F82130704740
:104E80001846704738B5437A994201D3002418E098
:104E9000036953F82140002243F82120002CF5D06B
:104EA0002378012B0DD9FFF763FF054628B10230A7
:104EB000A11C4FF4807203F037FD2378013B23706F
:104EC0002C46204638BD10B54168427A4B7A9A424A
:104ED0000ED872B60268D36813B9D06004E02346D6
:104EE000DC68002CFBD1D860012313720B7262B610
:104EF00010BDFFFF074B1A784AB9074AFF2111700E
:104F0000064A4FF080410120116018707047002060
:104F1000704700BF984400205EE400E008E100E034
:104F2000F8B5164B164D1A6842F080721A60154B90
:104F30001A6842F001021A60134B2E681C680FE0D9
:104F4000237A63B121682F680B68204698472A6846
:104F5000E388D21B12099A42A28088BFE28064696A
:104F6000002CEDD1064B094A1B689B1B1B091380C3
:104F7000074A11888B4288BF1380F8BDFCED00E022
:104F8000041000E0001000E08C440020B444002035
:104F90009A44002030B572B609B9026822B9264A8F
:104FA00000231188144611E003790F2BF7D822490A
:104FB000098841FA03F1C907F1D503F1007303F53C
:104FC0009063B2EB431FEAD162B630BD41FA03F2FF
:104FD00012F0010227D1012505FA03F529432180AA
:104FE00062B6164903710C6844F002040C6051F873
:104FF000044C44F0020441F8044C114982240C6032
:105000008B768B770B76CB7703F1007303F5906388
:105010005B0103601A605A609A60DA601A615A6133
:105020009A61DA6130BD0133102BCFD162B6002214
:105030000260037130BD00BFB844002040800440CE
:105040000080004003790F2B10D8094A137072B604
:10505000084B0279012101FA02F2198821EA0202C1
:105060001A8062B61023037100230360704700BFEB
:105070001A800040B844002008B5FCF723F8FBF77D
:1050800069FE00F0A3F9FAE7F8B506460C468F185A
:10509000002506E0336814F8011B1B68304698476A
:1050A0002D18BC42F6D12846F8BD2DE9F041002567
:1050B0008AB0074688468C682E4611E02B4640464B
:1050C00001A9212200F065F93B68202C34BF22465B
:1050D00020225B68384601A9AD18A41A98473618F3
:1050E000002CEBD130460AB0BDE8F08107B5054B86
:1050F0001B88ADF80430036801A95B680222984759
:105100000EBD00BFD89F0000F0B505468BB022B998
:105110000368C9B21B6898472CE0012A08BF0A221D
:1051200021B930228DF82520212413E02124B1FB60
:10513000F2F002FB1011C9B2092901D8303100E0A8
:1051400037310AAF3E1906F8241C014610B1013C64
:10515000E4B2ECE733B1013C0AAAE4B213192D2200
:1051600003F8242C2B6801AF5B6828463919C4F179
:10517000220298470BB0F0BD002902DA49422D23E4
:1051800000E000230A22FFF7BFBF08461146FFF7E1
:1051900001BD0846FFF766BDFFF76EBDFFF7CEBC49
:1051A000FFF7A4BCFFF7E8BC7047FFFF044B0022E9
:1051B0001A711A73034A4FF47A7199601A60704732
:1051C000BC440020E89F000010B5029C401AE41A7D
:1051D0004443521A94FBF2F0C01810BD10B50446B7
:1051E000006803F09BF8204610BD38B504460D4614
:1051F0000068013103F022FD10B184E82100012094
:1052000038BD43688B4210B5044600D306E0FFF773
:10521000ECFF20B1A3680BB922681370012010BD08
:10522000F8B504460F46154622B9036803B11A7053
:1052300000230BE01146FFF7E4FF064640B9206863
:1052400010B103F06BF8266000236360A36004E0F4
:10525000A5602068394604F063F82046F8BD38B5EB
:105260000023044603604360836003730D4639B135
:105270000846FEF747FD294602462046FFF7D0FFC5
:10528000204638BD81420B4603D009689A68FFF773
:10529000C7BF704738B505460C4641B10846FEF712
:1052A00031FD214602462846FFF7BAFF00E0A9601B
:1052B000284638BD10B5002386B00446036043601D
:1052C00083600373084601A9FEF742FD204601A949
:1052D000FFF7E0FF204606B010BD70B504460E464D
:1052E00085685AB155192946FFF78BFF30B1206800
:1052F000A3683146C01804F013F8A560204670BDBD
:105300000B4609689A68FFF7E8BF38B505460C46B2
:1053100039B10846FEF7F6FC214602462846FFF75B
:10532000DCFF284638BD10B58B688468E41AA242B9
:105330000CD8006868B1096851B180181A4604F0A9
:105340004DF8D0F1010038BF002010BD002010BD85
:10535000084610BD82688B689A4202D30022FFF78C
:10536000E2BF0020704708B582688B689A420CD370
:10537000006868B1096851B1D31AC01803F0E2FEA1
:10538000D0F1010038BF002008BD002008BD08464C
:1053900008BD38B50C469AB191B181688B4202D3F1
:1053A0000023237038BDCD1A013A0168954228BF09
:1053B0001546C91820462A4604F066F800236355AE
:1053C00038BD006808B102F05DBF704708B50E4BEC
:1053D0001A78C2B901221A70FFF7CEFB08B1FFF7A5
:1053E000E3FE00F08BF908B100F0E6FE00F0C4FB2C
:1053F00008B100F053FF00F0A9FD08B100F0C0FFB4
:10540000014B00221A7008BDCC440020194B1A68C9
:1054100042F480621A60184A00231370174A13700E
:10542000174A1370174A1370174A1370174B40F23C
:1054300013321A604FF451725A60154BC0F3443264
:105440001A70C0F347125A700221042200F01F00A4
:1054500098729A70D9745A7588221A743C22DA703C
:105460000C4B40226FF44A711A705B184FF40052D3
:105470001A607047348004404F450020CE4400201D
:105480005845002050450020CD44002040A0044055
:1054900000A006402DE400E0134A937800F00301D9
:1054A00003F0EC030B43410748BF43F01003937034
:1054B00000F00F03042B0C4903D18B7943F0400318
:1054C0008B715379C20603F0EF03074A48BF43F0DC
:1054D000100353719379800603F0EF0348BF43F044
:1054E00010039371704700BF00A006400E4B1B686D
:1054F000580510B503D410BDFFF768FF00E00B4C52
:105500002378002BF8D10A4A4FF400511160094A60
:105510000949D37040F203120A604A60074A1370C7
:10552000074A137010BD00BF34800440CD440020F2
:1055300084E100E000A0064040A004404F45002068
:10554000CE44002038B5094B04461D78002DFCD10F
:1055500020460121FEF7C2FD20462946FEF792FDB6
:10556000034B53F83420034B1A6038BDCD44002060
:10557000C89E0000544500201D4B1B685A052DE9AC
:10558000F041074631D51B4B1B680BB101221A7045
:10559000194B1A4D1C781A4EDFF8688001343F2CE5
:1055A00088BF002414E0FEF78FFB40280CDC337921
:1055B0001B060DD52B7801333F2B88BF002318F82D
:1055C0000320F2712B7003E0FF2801DDFFF7FEFEE0
:1055D0002B78A342E7D00B4B1F550B4B01221A70BF
:1055E000054B1C70064BBC22DA70BDE8F08100BF91
:1055F0003480044054450020584500205045002088
:1056000000A00640CF440020CD4400202DE9F84FF3
:10561000254B1B6806465805894642D5234B1B6817
:105620000BB101221A70224DB346AA4632E0214B3B
:105630001C782F7801343F2C88BF0024A74209D062
:105640001BF8012B1C4B1A551C4B01221A70194BCD
:105650001C701FE01A4BBC22DA709846FEF734FB30
:1056600040280FDC98F8043019060FD52B78124A21
:1056700001333F2B88BF0023D25C88F807208AF8CB
:10568000003003E0FF2801DDFFF7A0FE2B78BB42CE
:10569000E4D0D5E706EB09039B45C8D3084BBC22F1
:1056A000DA70BDE8F88F00BF348004405445002014
:1056B0005045002058450020CF440020CD44002014
:1056C00000A0064010B5044C01E0FFF77FFE2378F0
:1056D000002BFAD110BD00BFCD440020054B064A77
:1056E0001B781078834201D33F3000E00138C01AA4
:1056F000704700BF5845002050450020044B1878E3
:10570000044B1B78984238BF4030C01A704700BF26
:105710004F450020CE440020084B094A19781378E1
:10572000994207D001333F2B88BF00230549C85C4D
:10573000137070474FF0FF30704700BF4F45002097
:10574000CE4400200F450020074B1A78074B1B78EA
:105750009A4206D001333F2B88BF0023044AD05C15
:1057600070474FF0FF3070474F450020CE44002077
:105770000F450020094B1B685B050ED5084BDA78F6
:1057800002F0CB02DA7040225A74DA7842F0340226
:10579000DA70044B1A78044B1A7070473480044056
:1057A00000A00640CE4400204F45002070B52D4B90
:1057B0001A7912F0300F1DD072B6997D21B9DA79BD
:1057C00040225A7462B615E062B6274A274812781A
:1057D000274D00781C46531C3F2B88BF0023E679D9
:1057E00083421CBFEE541A46013911F0FF01F2D179
:1057F0001D4B1A701B4AD37819465BB2002B1BDA7B
:105800001379180618D51B4B1B4C1D781B4B1B78A6
:10581000AB4209D001333F2B88BF00231079E05CF5
:10582000D071107D0728F3D9144A13700D4B1A79E3
:10583000120601D57C22DA7001F04003DBB27BB1A5
:10584000084B1A7902F04002D2B2194642B10C4B11
:1058500000221A700B4B1B6803B11A703C23CB70EB
:1058600070BD00BF00A006404F450020CE44002080
:105870000F45002058450020CF440020504500200F
:10588000CD44002054450020184B1A6842F40062B1
:105890001A60174A00231370164A1370164A1370C1
:1058A000164A1370164A1370164B40F213321A60E0
:1058B0004FF451725A60144BC0F344321A70C0F363
:1058C00047125A7000F01F000422022198729A7049
:1058D000D9745A7588221A743C22DA700B4B402214
:1058E0001A700B4B4FF400421A607047348004402A
:1058F000C34500205A450020CC450020C445002067
:10590000594500200CB0044000B006402FE400E0F0
:1059100004E100E0134A937800F0030103F0EC0384
:105920000B43410748BF43F01003937000F00F038F
:10593000042B0C4903D18B7943F040038B715379CD
:10594000C20603F0EF03074A48BF43F01003537148
:105950009379810603F0EF0348BF43F0100393717E
:10596000704700BF00B006400E4B1B68180510B50D
:1059700003D410BDFFF72AFD00E00B4C2378002B69
:10598000F8D10A4A4FF400411160094A0949D3701D
:1059900040F203120A604A60074A1370074A137004
:1059A00010BD00BF348004405945002084E100E070
:1059B00000B006400CB00440C34500205A4500200A
:1059C00038B5094B04461D78002DFCD12046012135
:1059D000FEF784FB20462946FEF754FB034B53F8A1
:1059E0003420034B1A6038BD59450020C89E000082
:1059F000C84500201D4B1B681A052DE9F0410746DC
:105A000031D51B4B1B680BB101221A70194B1A4D73
:105A10001C781A4EDFF868800134272C88BF0024D8
:105A200014E0FEF751F940280CDC33791B060DD544
:105A30002B780133272B88BF002318F80320F2713D
:105A40002B7003E0FF2801DDFFF7C0FC2B78A34299
:105A5000E7D00B4B1F550B4B01221A70054B1C70E6
:105A6000064BBC22DA70BDE8F08100BF34800440F0
:105A7000C8450020CC450020C445002000B00640A9
:105A80005B450020594500202DE9F84F254B1B6848
:105A900006461805894642D5234B1B680BB10122E7
:105AA0001A70224DB346AA4632E0214B1C782F785B
:105AB0000134272C88BF0024A74209D01BF8012BF2
:105AC0001C4B1A551C4B01221A70194B1C701FE0FD
:105AD0001A4BBC22DA709846FEF7F6F840280FDC25
:105AE00098F8043019060FD52B78124A0133272B6A
:105AF00088BF0023D25C88F807208AF8003003E0D2
:105B0000FF2801DDFFF762FC2B78BB42E4D0D5E72C
:105B100006EB09039B45C8D3084BBC22DA70BDE8ED
:105B2000F88F00BF34800440C8450020C4450020E1
:105B3000CC4500205B4500205945002000B00640C0
:105B400010B5044C01E0FFF741FC2378002BFAD19B
:105B500010BD00BF59450020054B064A1B78107840
:105B6000834201D3273000E00138C01A704700BFDC
:105B7000CC450020C4450020044B1878044B1B780A
:105B8000984238BF4030C01A704700BFC34500205C
:105B90005A450020084B094A19781378994207D0D2
:105BA00001333F2B88BF00230549C85C1370704741
:105BB0004FF0FF30704700BFC34500205A4500201A
:105BC00083450020074B1A78074B1B789A4206D072
:105BD00001333F2B88BF0023044AD05C70474FF04D
:105BE000FF307047C34500205A4500208345002000
:105BF000094B1B681B050ED5084BDA7802F0CB0267
:105C0000DA7040225A74DA7842F03402DA70044BC7
:105C10001A78044B1A7070473480044000B0064074
:105C20005A450020C345002070B52D4B1A7912F05B
:105C3000300F1DD072B6997D21B9DA7940225A749D
:105C400062B615E062B6274A27481278274D0078D9
:105C50001C46531C3F2B88BF0023E67983421CBFA0
:105C6000EE541A46013911F0FF01F2D11D4B1A70A2
:105C70001B4AD37819465BB2002B1BDA137918063E
:105C800018D51B4B1B4C1D781B4B1B78AB4209D006
:105C90000133272B88BF00231079E05CD071107D81
:105CA0000728F3D9144A13700D4B1A79120601D53F
:105CB0007C22DA7001F04003DBB27BB1084B1A7929
:105CC00002F04002D2B2194642B10C4B00221A70C7
:105CD0000B4B1B6803B11A703C23CB7070BD00BF27
:105CE00000B00640C34500205A45002083450020EF
:105CF000CC4500205B450020C445002059450020CC
:105D0000C8450020174B1A6842F480521A60164AA0
:105D100000231370154A1370154A1370154A137037
:105D2000154A1370154A40F2133111604FF4517146
:105D30005160134AC0F344311170C0F3471100F0B1
:105D40001F0051709072937013742C23D3700D4BFD
:105D500040226FF44B711A705B184FF400321A60D6
:105D6000704700BF3480044037460020CE450020F5
:105D70004046002038460020CD45002008C00440A1
:105D800000C0064031E400E0134A937800F00301BC
:105D900003F0EC030B43410748BF43F0100393703B
:105DA00000F00F03042B0C4903D18B7943F040031F
:105DB0008B715379C20603F0EF03074A48BF43F0E3
:105DC000100353719379800603F0EF0348BF43F04B
:105DD00010039371704700BF00C006400E4B1B6854
:105DE000D80410B503D410BDFFF7F0FA00E00B4C57
:105DF0002378002BF8D10A4A4FF400311160094A88
:105E00000949D37040F203120A604A60074A1370CE
:105E1000074A137010BD00BF34800440CD450020F8
:105E200084E100E000C0064008C00440374600207E
:105E3000CE45002038B5094B04461D78002DFCD115
:105E400020460121FEF74AF920462946FEF71AF9B5
:105E5000034B53F83420034B1A6038BDCD45002066
:105E6000C89E00003C4600201D4B1B68DA042DE94B
:105E7000F041074631D51B4B1B680BB101221A704C
:105E8000194B1A4D1C781A4EDFF868800134272C04
:105E900088BF002414E0FDF717FF40280CDC33799D
:105EA0001B060DD52B780133272B88BF002318F84C
:105EB0000320F2712B7003E0FF2801DDFFF786FA63
:105EC0002B78A342E7D00B4B1F550B4B01221A70C6
:105ED000054B1C70064BAC22DA70BDE8F08100BFA8
:105EE000348004403C4600204046002038460020D4
:105EF00000C00640CF450020CD45002038B54518EC
:105F0000044603E014F8010BFFF7AEFFAC42F9D1F1
:105F100038BDFFFF10B5044C01E0FFF757FA2378B6
:105F2000002BFAD110BD00BFCD450020054B064A1D
:105F30001B781078834201D3273000E00138C01A63
:105F4000704700BF4046002038460020044B1878B8
:105F5000044B1B78984238BF4030C01A704700BFCE
:105F600037460020CE450020084B094A197813789F
:105F7000994207D001333F2B88BF00230549C85CF5
:105F8000137070474FF0FF30704700BF3746002056
:105F9000CE450020F7450020074B1A78074B1B78A9
:105FA0009A4206D001333F2B88BF0023044AD05CBD
:105FB00070474FF0FF30704737460020CE45002035
:105FC000F7450020024B1A78024B1A70704700BF49
:105FD000CE4500203746002010B5214B1A7902F03B
:105FE0002002D2B26AB11F4AD8791F4913780978C2
:105FF00001333F2B88BF00238B4202D01B49C8547A
:106000001370174AD37818465BB2002B13DA137952
:10601000190610D5164B17491C780B789C4202D1F3
:106020006C23D37007E00133272B88BF0023124C69
:10603000E45CD4710B7000F04003DBB27BB1084B21
:106040001A7902F04002D2B2194642B10B4B00223B
:106050001A700B4B1B6803B11A702C23CB7010BD48
:1060600000C0064037460020CE450020F7450020FE
:106070004046002038460020CF450020CD45002076
:106080003C4600201FB572B6154B70221A70154A97
:10609000412111700F2102F8011C80221A701A7818
:1060A0001206FCD5104B186862B6104B984201D806
:1060B0000A23584301A90A22FDF72CFE0C480023AD
:1060C00001AA9A5C2AB100EB430101330A2B4A80F2
:1060D000F6D10133064A5B00137005B000BD00BF66
:1060E0000000024007000240080002407F9698002E
:1060F0000890FF1F08B50368C9B21B68984708BD20
:1061000008B50368C9B21B68984708BD08B503689D
:10611000C9B21B68984708BD08B50368C9B21B68B7
:10612000984708BD084608B5FFF726FA012008BDC4
:10613000084608B5FFF720FA012008BD38B5084623
:106140000D46FDF7DFFD044621462846FFF75EFABF
:10615000204638BD10B5084614461146FFF756FADA
:10616000204610BDFFF7BABAFFF704BBFFF7AABA83
:10617000FFF7D2BAFFF7E8BAFFF7C0BA0846FFF751
:10618000E1B9FFF7B3B9480800F1376000F5D8303E
:10619000B0FBF1F0FFF73AB9480800F1376010B5ED
:1061A00000F5D830B0FBF1F01446FFF72FF9204688
:1061B000BDE81040FFF770B97047FFFF044B0022A5
:1061C0001A711A73034A4FF47A7199601A60704712
:1061D0004446002060A0000008B50368C9B21B68EF
:1061E000984708BD08B50368C9B21B68984708BD41
:1061F00008B50368C9B21B68984708BD08B50368AD
:10620000C9B21B68984708BD084608B5FFF7F2FBFE
:10621000012008BD084608B5FFF7ECFB012008BDCA
:1062200038B508460D46FDF76DFD04462146284663
:10623000FFF72AFC204638BD10B508461446114623
:10624000FFF722FC204610BDFFF786BCFFF7D0BC4D
:10625000FFF776BCFFF79EBCFFF7B4BCFFF78CBC22
:106260000846FFF7ADBBFFF77FBB480800F137607A
:1062700000F5D830B0FBF1F0FFF706BB480800F19D
:10628000376010B500F5D830B0FBF1F01446FFF7D9
:10629000FBFA2046BDE81040FFF73CBB7047FFFF0C
:1062A000044B00221A711A73034A4FF47A719960F1
:1062B0001A60704754460020B0A0000008B503687B
:1062C000C9B21B68984708BD08B50368C9B21B6806
:1062D000984708BD08B50368C9B21B68984708BD50
:1062E00008B50368C9B21B68984708BD084608B5D9
:1062F000FFF7BAFD012008BD084608B5FFF7B4FD59
:10630000012008BD38B508460D46FDF7FBFC0446E4
:1063100021462846FFF7F2FD204638BD10B5084655
:1063200014461146FFF7EAFD204610BDFFF7FEBDFB
:10633000FFF748BEFFF7EEBDFFF716BEFFF72CBE16
:10634000FFF704BE0846FFF775BDFFF747BD4808D5
:1063500000F1B76000F55840B0FBF1F0FFF7D2BC98
:10636000480800F1B76010B500F55840B0FBF1F0F7
:106370001446FFF7C7FC2046BDE81040FFF704BDF8
:106380007047FFFF044B00221A711A73034A4FF43F
:106390007A7199601A6070476446002000A100007D
:1063A0002DE9F04F8BB01F4680468946164600F017
:1063B00093F949F21E0BC1F6FF7B9BF900300133C4
:1063C00004460D4604D03046394600F0F5FF20B9AA
:1063D000204629460BB0BDE8F08F4046494600F004
:1063E000EBFF824620BB304639460022002301F0F5
:1063F00059FD0028ECD09BF900104AF24813012205
:10640000C0F200038DE80C0000220023B1F1FF3F31
:1064100018BF0229C3F6F073CDF820A0CDE9028998
:10642000CDE90467CDE906232DD1DDE90645CFE7A7
:10643000404649460022002301F034FD00282FD0B9
:10644000304639460022002301F02CFD002861D09F
:106450009BF900204AF24813C0F2000301210020FA
:106460008DE80A00CDE90289002300210893CDE9D7
:106470000467CDE9060132B100230022C3F6F073B0
:10648000CDE90623D1E7684600F0BEFF002870D0B2
:10649000089B002BC9D001F007FF089B0360C4E7ED
:1064A0002046294600F082FF8246002866D020461A
:1064B00029460022002301F0F5FC002888D0404640
:1064C000494600F073FF002882D03046394600F07C
:1064D0006DFF00283FF47CAF9BF900204AF248137F
:1064E0000421C0F2000300208DE80A0000230021EF
:1064F000022A0893CDE90289CDE90467CDE90601B6
:1065000069D0684600F080FF002864D0089B002B0B
:106510008BD0C0E73046394600F048FF00283FF4F2
:1065200057AF304639460022002301F0C5FC002851
:106530003FF44EAF9BF800104AF24813C0F200033C
:106540000122CDE902898DE80C000023CDE9046722
:10655000002208930023002936D1CDE9062368469E
:1065600000F052FF0028D1D101F09EFE21230360EC
:10657000CCE701F099FE2123036089E740464946B4
:1065800000F014FF002892D03046394600F00EFF8C
:1065900000288CD02046294600F00EFF00BB9BF857
:1065A00000404AF24813C0F2000301220890002183
:1065B0008DE80C000020CDE90289CDE90467002CAC
:1065C00063D1CDE90601CAE70229CFF6F073CDE920
:1065D0000623C9D0C3E701F067FE2223036095E7D5
:1065E0009BF900104AF248120320C0F20002CDF8D5
:1065F00020A08DE805004046CDE90289CDE9046779
:10660000E9B94FF6FF754946002200234FF0604478
:10661000C4F2EF75CDE9064501F04EFC00283ED1ED
:106620009BF90030022B05D0684600F0EDFE0028F3
:106630007FF42EAF01F038FE2223036028E7002507
:106640004946002200230024C7F6F075CDE906452F
:1066500001F032FC0028E3D000230022C3F6E073EF
:106660003046394601F0B6F904460D4600F0D4FE36
:1066700022462B4601F016FC0028D1D1002300222F
:10668000CFF6F073CDE90623CAE702460B4601F0C8
:10669000CBFA022CCDE906013FF466AF5FE7002399
:1066A0000022C3F6E0733046394601F093F9044600
:1066B0000D4600F0B1FE22462B4601F0F3FB002808
:1066C000AED14FF6FF734FF06042CCF2EF73CDE9DD
:1066D0000623A5E7FFFFFFFF2DE9F04F91B023F060
:1066E00000478B460D46049157EA020191468246C7
:1066F0001E4604469446804600F08E8000212BF012
:106700000040C7F6F0710290884211DD029901F154
:10671000404909F5801959EA080840F082800026AE
:10672000C146C3F6F0764846314611B0BDE8F08F59
:1067300014BF002001200690BAF1000F0CBF00200A
:1067400000F001000028E1D18F42DFDC14BF0020FF
:106750000120002A0CBF002100F001010029D5D141
:10676000049A5C461D46002A64DB0E91BCF1000FC2
:1067700014D1002840F082800023C3F6F0739F42BA
:1067800000F0B880B5F1804F04BF504659463CD068
:106790000023C3F6E0739D4200F0C0835046594683
:1067A00000F000FE8C46B8F1000F0BD1069B029959
:1067B000002908BF43F00103002B76D1C3F6F07324
:1067C000994272D0049B0E994FEAD37808F1FF38B2
:1067D00051EA080100F089800023C4F2E0139F42CF
:1067E00040F3A6800023C4F2F0339F4240F330848C
:1067F0004FF6FF73029AC3F6EF739A4240F39E83FB
:10680000002D4EDD48A1D1E9000102460B4601F002
:10681000E1F881460E4686E700268946C3F6F07603
:1068200081E74AF28010C0F2000011B0BDE8F04FDD
:1068300000F0ECBD4FF6FF73C4F23F339F426ADCB9
:106840004FF6FF73C3F6EF739F428EDD3B1540F2A8
:106850001342934240F38B84C3F5866303332CFACF
:1068600003F202FA03F3634502BF02F00103C3F12E
:1068700002030E933FF47AAF002176E7029A02F109
:10688000404303F5801353EA080300F051834FF6A9
:10689000FF73C3F6EF739A4240F3B283002DBFF645
:1068A00042AF4FF000094E463DE7002DA8BF6646B7
:1068B000C0F24284002CA8BF8146BFF634AF029AD2
:1068C0000E9902F1404303F58013194340F05F84B1
:1068D000804602463346314600F0C8FE02460B466B
:1068E00001F0A2F981460E461DE750465946524630
:1068F0005B46F1E7002DA4BFD1465E46BFF613AF5D
:10690000002152460020C3F6F0715B4601F08CF97D
:1069100081460E4607E702230E93BCF1000F3FF4B9
:1069200028AF3BE7AFF300809C7500883CE4377EDE
:10693000029B0021B3F5801F0BDA00236146002281
:10694000C4F2403301F046F88C466FF03401CDF8C4
:1069500008C0029A002522F07F43141549F68E02E2
:1069600023F47003C0F20302934243F07F57A4F272
:10697000FF340C440F9447F440142F460FDD4BF2C4
:1069800079620127C0F20B024FF48025934206DDA5
:1069900000250F9BA4F580142F4601330F934AF274
:1069A00050110246C0F20001234601EBC707CDE9B2
:1069B0000823D7E90001CDE90A0110462146DDE9A7
:1069C0000A2300F053FEDDE90A2382468B46DDE907
:1069D000080100F04DFE0B4600210246C3F6F0719F
:1069E000002001F021F9CDE90C015046DDE90C232E
:1069F000594600F0EFFFCDE906016110DDE90623FD
:106A000041F00051002001F50021CDE904236B186D
:106A100004900022DDE9040114461D46CDE902017F
:106A200000F0D8FF02460B465046594600F01EFEC5
:106A3000DDE90A2382468B462046294600F016FEF1
:106A400002460B46DDE9080100F010FE02460B4647
:106A5000DDE9020100F0BEFF02460B4650465946F2
:106A600000F004FEDDE90C2300F0B4FF82468B4603
:106A7000DDE9060102460B4600F0ACFF02460B467C
:106A800004460D4600F0A6FFA3A3D3E90023CDE9F9
:106A900008012046294600F09DFFA1A3D3E9002369
:106AA00000F0E6FD22462B4600F094FF9EA3D3E9BA
:106AB000002300F0DDFD22462B4600F08BFF9CA357
:106AC000D3E9002300F0D4FD22462B4600F082FFDC
:106AD00099A3D3E9002300F0CBFD22462B4600F01A
:106AE00079FF97A3D3E9002300F0C2FD02460B46CD
:106AF000DDE9080100F06EFFDDE9062304460D46DE
:106B0000DDE9020100F0B4FD52465B4600F062FF91
:106B100022462B4600F0ACFDCDE90801DDE902017B
:106B200002460B4600F056FF00220023C4F2080381
:106B3000CDE90A0100F09CFDDDE9082300F098FD95
:106B40000D4604992B460C46DDE90201224600F071
:106B500041FF22462B46CDE902015046594600F03E
:106B600039FF00230022C4F2080382468B462046E8
:106B7000294600F07BFDDDE90A2300F077FD02469F
:106B80000B46DDE9080100F071FDDDE9062300F0A8
:106B900021FF02460B465046594600F069FD8246E9
:106BA0008B4652465B46DDE9020100F061FD049A26
:106BB000104665A3D3E9002304460D4600F00AFF02
:106BC00063A3D3E90023CDE906012046294600F05E
:106BD00001FFDDE90223CDE908012046294600F046
:106BE00045FD02460B465046594600F03FFD5AA36C
:106BF000D3E9002300F0EEFE02460B46DDE9080172
:106C000000F036FDD7E9042300F032FD82460F98EC
:106C10008B4600F079FE52465B4604460D46D7E9A6
:106C20000801CDE90201DDE9060100F021FDDDE901
:106C3000022300F01DFD22462B4600F019FD049AA8
:106C40002B461046224604460D4600F00FFDDDE9B6
:106C5000022300F00BFDDDE9062300F007FD0246EC
:106C60000B465046594600F001FD82468B460E9871
:106C7000431E53EA080340F0BC8100230022CBF6F8
:106C8000F073CDE904233346002231464846CDE96E
:106C9000022300F0EBFC22462B4600F09BFE5246FE
:106CA0005B46CDE906013146484600F093FE0246B8
:106CB0000B46DDE9060100F0DBFC22462B4682464E
:106CC0008B46DDE9020100F085FE04460D46504684
:106CD000594622462B4600F0CBFC4FF6FF7CC4F20F
:106CE0008F0C614506460F46884640F32B8101F123
:106CF0003F4303F5E003034340F0298218A3D3E99F
:106D000000235046594627F0004900F0B1FC2246C6
:106D10002B46CDE9020127E0EF4E454A287ECA3FC7
:106D200065DBC9934A86CD3F01411DA96074D13FFF
:106D30004D268F515555D53FFFAB6FDBB66DDB3F11
:106D4000033333333333E33F000000E009C7EE3F42
:106D5000F5015B14E02F3EBEFD033ADC09C7EE3FB0
:106D6000FE822B654715973C3046394600F07EFC85
:106D700002460B46DDE9020101F0BCF8002840F0B4
:106D8000E6810023C3F6E0739945DCBF4FF0000CA9
:106D9000CDF808C000F3F48000269DA3D3E90023BA
:106DA00030463946CDF804C000F014FE22462B468A
:106DB000804689463046394600F058FC02460B466C
:106DC0005046594600F052FC93A3D3E9002300F04B
:106DD00001FE93A3D3E9002304460D46304639460D
:106DE00000F0F8FD02460B462046294600F040FC24
:106DF00004460D4622462B464046494600F038FCE4
:106E000042464B4682468B4600F030FC02460B461B
:106E10002046294600F02AFC52465B4680468946B9
:106E20005046594600F0D6FD7FA3D3E9002304461F
:106E30000D4600F0CFFD7EA3D3E9002300F016FC41
:106E400022462B4600F0C6FD7BA3D3E9002300F0C9
:106E50000FFC22462B4600F0BDFD79A3D3E90023A9
:106E600000F004FC22462B4600F0B4FD76A3D3E9E3
:106E7000002300F0FDFB22462B4600F0ABFD02464E
:106E80000B465046594600F0F1FB04460D4622469B
:106E90002B465046594600F09DFD00224FF080439E
:106EA00006460F462046294600F0E0FB02460B4608
:106EB0003046394600F0B8FE42464B4604460D4681
:106EC0005046594600F086FD42464B4600F0D0FB46
:106ED00002460B462046294600F0C8FB52465B4658
:106EE00000F0C4FB0B4600210246C3F6F0710020FF
:106EF00000F0BCFBDDF804C00CEB01040B46B4F55C
:106F0000801F02460D46A8BF2346C0F25E81DDE920
:106F1000040100F05FFD81460E4604E4002CFFF6FC
:106F20003DAC5046594611B0BDE8F04F00F074B981
:106F300000269946C3F6F076FFF7F5BB002DBFF6A5
:106F4000B0AC5FE44CF6FF3321F00049C4F290038B
:106F500099457FF716AF4FF45053C3F66F73CB18B4
:106F6000034340F01A8122462B4600F07FFB024685
:106F70000B465046594600F0A9FF002840F00D810D
:106F80004FEA29534FF48011A3F2FE334FF6FF76F8
:106F900041FA03F1C0F20F064144002221F07F477D
:106FA000C1F30A5027F47007A0F2FF3E47F48017A0
:106FB000C0F58260B8F1000F46FA0EF600F1030C3E
:106FC00021EA060347FA0CFCCDF808C0C0F2F980AC
:106FD0002046294600F04AFB04460D46224650460C
:106FE00059462B4600F044FB029A4FEA025C0F46DA
:106FF000D2E600210020C3F6F071CDE9040142E69B
:10700000002DBFF64EAC06F10046FFF78CBB00BF6B
:1070100000000000432EE63FEF39FAFE422EE63F25
:10702000396CA80C615C20BED0A4BE726937663E84
:10703000F16BD2C541BDBB3E2CDE25AF6A56113F78
:1070400093BDBE166CC1663F3E5555555555C53F5F
:107050004FF6FE730299C3F6EF7399427FF76EAF56
:107060000023029AC3F6F0739A423FF7C9AB00239C
:1070700061460022C3F6F07300F0F8FA5AA3D3E990
:10708000002304460D4600F0A5FC59A3D3E90023D4
:1070900082468B462046294600F09CFC22462B4621
:1070A000CDE902012046294600F094FC002300228D
:1070B000C3F6D073CDE904012046294600F08AFCCE
:1070C00002460B464CA1D1E9000100F0CFFA22465E
:1070D0002B4600F07FFC0B4600210246C3F6E07110
:1070E000002000F0C3FA02460B46DDE9040100F07F
:1070F00071FC43A3D3E9002300F06CFC02460B466D
:10710000DDE9020100F0B2FACDE902015046DDE905
:107110000223594600F0ACFA52465B460020044672
:107120000D4600F0A3FA02460B46DDE9020100F02D
:107130009DFA82468B469AE500210246C3F6F0711D
:107140000020634600F070FD0E46FFF7B3BB2EA390
:10715000D3E90023DDE9040100F03CFC2AA3D3E9D4
:10716000002300F037FC81460E46FFF7DCBABCF185
:10717000000F22D1C3F58263DA1C47FA02F303FA47
:1071800002F2BA4227D000230E93FFF7F2BA0E9A0A
:107190008146012A7FF4C7AA35E71DA3D3E900235E
:1071A000DDE9040100F016FC19A3D3E9002300F087
:1071B00011FC81460E46FFF7B6BA00230E93FFF787
:1071C000EDBA61464942029102E7029A00F0BCF929
:1071D00002460B469BE603F00103C3F102030E9344
:1071E000FFF7C7BAAFF30080000000604715F73F14
:1071F00044DF5DF80BAE543E555555555555D53FBA
:10720000FE822B654715F73F9C7500883CE4377E6E
:1072100059F3F8C21F6EA5012DE9F8430027B946BE
:10722000C7F6F077C7F6F0790F404F4504460D4694
:1072300002460B460E46804600F09980002977DD15
:107240000F1500F0828026F07F43A7F2FF3723F46A
:107250007003FA0743F4801344BF4FEAD8724FEA31
:1072600048084FF0000C48BF02EB430360464FEA6A
:10727000D8727F1002EB430316244FEA48024FF402
:1072800000114518D60F9D424FEA4202DEBFC5EB02
:10729000030368188C444908013C06EB4303F0D112
:1072A0002026A0464FF000410EE081461B1A954271
:1072B00088BF013B521B64184846D50F490852004D
:1072C000013E05EB430315D0984201EB080503DBB3
:1072D000954298BF8342F0D105F0004905EB0108C3
:1072E000B9F1004FE1D1B8F1000FA8BF00F10109D9
:1072F000DCDADAE7134312D166084FEA6C031CF0BC
:10730000010F03F17F5318BF46F0004603F5001349
:10731000344603EB075520462946BDE8F883631C35
:1073200008BF0CF1010CE8D004F001031C19E3E7DD
:1073300021F000460643EED041BB0F464FEAD82667
:10734000153F4FEA4858002EF8D016F4801319D193
:1073500076000133F102FBD5C3F10101C3F1200234
:1073600028FA02F27F18164308FA03F86BE700F0D8
:1073700031FB02460B462046294600F079F90446C7
:107380000D46C8E7202201210023E9E702460B460B
:1073900000F06CF902460B4600F046FC04460D4630
:1073A000B9E700BF21F00041704700BF41F0004144
:1073B00001F58010C00F704750EA010201D1022090
:1073C0007047D0F1010238BF0022B1F1004F08BF71
:1073D0000028F4D021F000434FF6FF71A3F5801090
:1073E000C7F6DF71884201D804207047B3F5801FCB
:1073F00001D2032070470020C7F6F070834214BF0B
:10740000002002F00100704700207047002100209A
:10741000C7F6F871704700BFC1F30A5C02462DE958
:10742000F041ACF2FF36CD0F132E82B00B4604466E
:107430000F4688463ADC002E56DB4FF6FF71C0F24D
:107440000F0141FA06F101EA0300104329D049086F
:107450000B4053EA02040CD04FF4802327EA0108C2
:10746000132E0CBF4FF00044002443FA06F648EAFE
:1074700006084AF288112246C0F20001434601EB99
:10748000C505D5E900452046294600F0F1F8224619
:107490002B46CDE90001DDE9000100F0E7F80246E6
:1074A0000B461046194602B0BDE8F081332E07DDC9
:1074B000B6F5806FF5D100F0DBF802460B46F0E739
:1074C0004FF0FF31ACF2134C21FA0CF10142E8D03D
:1074D000490801421FBF4FF0804320EA010443FAEC
:1074E0000CFC44EA0C04C4E721F000410143D8D06D
:1074F00023F07F404AF2881120F47000C0F20001AE
:1075000040EA020401EBC50160424FEA534E0443D6
:10751000D1E90067240B304604F40024394644EADC
:107520004E4300F0A5F832463B46CDE90001DDE9C7
:10753000000100F09BF80F4621F00041064602468C
:1075400041EAC573ADE700BFC1F30A532DE9F0412D
:1075500004460D46904606460F46C3B921F0004C3E
:107560005CEA000C29D000230022C4F2503300F062
:1075700031FA43F6B043CFF6FF73984504460D4603
:1075800006460F462BDBC1F30A53363B05E040F2BB
:10759000FF72934218BF094636D0434440F2FE7250
:1075A0009342C4BF22462B4621DC002B09DD21F08B
:1075B000FF4121F4E00141EA035520462946BDE898
:1075C000F08113F1350F26DA4CF2503322469845FC
:1075D0002B460CDC1AA1D1E9000100F039F818A300
:1075E000D3E9002300F0F6F904460D46E5E716A1BD
:1075F000D1E9000100F02CF813A3D3E9002300F037
:10760000E9F904460D46D8E72B46024600F030F86B
:1076100004460D46D1E7363321F0FF4121F4E00165
:10762000204641EA0355002329460022C3F6904331
:1076300000F0D0F904460D46BFE700BFAFF300806D
:1076400059F3F8C21F6EA5019C7500883CE4377E93
:1076500010B421F0004203F0004444EA020110BCDF
:10766000704700BF81F0004102E000BF83F000439B
:1076700030B54FEA41044FEA430594EA050F08BFCD
:1076800090EA020F1FBF54EA000C55EA020C7FEA91
:10769000645C7FEA655C00F0E2804FEA5454D4EB0E
:1076A0005555B8BF6D420CDD2C4480EA020281EAD8
:1076B000030382EA000083EA010180EA020281EA10
:1076C0000303362D88BF30BD11F0004F4FEA013162
:1076D0004FF4801C4CEA113102D0404261EB410171
:1076E00013F0004F4FEA03334CEA133302D05242F7
:1076F00063EB430394EA050F00F0A780A4F10104B3
:10770000D5F1200E0DDB02FA0EFC22FA05F28018EC
:1077100041F1000103FA0EF2801843FA05F35941D2
:107720000EE0A5F120050EF1200E012A03FA0EFC51
:1077300028BF4CF0020C43FA05F3C01851EBE3717B
:1077400001F0004507D54FF0000EDCF1000C7EEB98
:1077500000006EEB0101B1F5801F1BD3B1F5001FD6
:107760000CD349085FEA30004FEA3C0C04F10104F5
:107770004FEA445212F5800F80F09A80BCF1004F1E
:1077800008BF5FEA500C50F1000041EB045141EAA0
:10779000050130BD5FEA4C0C404141EB010111F4A1
:1077A000801FA4F10104E9D191F0000F04BF01464C
:1077B0000020B1FA81F308BF2033A3F10B03B3F12A
:1077C00020020CDA0C3208DD02F1140CC2F10C02BA
:1077D00001FA0CF021FA02F10CE002F11402D8BF18
:1077E000C2F1200C01FA02F120FA0CFCDCBF41EAE4
:1077F0000C019040E41AA2BF01EB0451294330BDB3
:107800006FEA04041F3C1CDA0C340EDC04F114048F
:10781000C4F1200220FA04F001FA02F340EA030066
:1078200021FA04F345EA030130BDC4F10C04C4F1AC
:10783000200220FA02F001FA04F340EA030029468C
:1078400030BD21FA04F0294630BD94F0000F83F4D6
:10785000801306BF81F480110134013D4EE77FEAB9
:10786000645C18BF7FEA655C29D094EA050F08BF05
:1078700090EA020F05D054EA000C04BF19461046E6
:1078800030BD91EA030F1EBF0021002030BD5FEA2A
:10789000545C05D14000494128BF41F0004130BD52
:1078A00014F580043CBF01F5801130BD01F00045A6
:1078B00045F0FE4141F470014FF0000030BD7FEA19
:1078C000645C1ABF194610467FEA655C1CBF0B4614
:1078D000024650EA013406BF52EA033591EA030F2B
:1078E00041F4002130BD00BF90F0000F04BF002123
:1078F000704730B54FF4806404F132044FF0000556
:107900004FF0000150E700BF90F0000F04BF0021CE
:10791000704730B54FF4806404F1320410F0004534
:1079200048BF40424FF000013EE700BF42004FEA2F
:10793000E2014FEA31014FEA02701FBF12F07F43AC
:1079400093F07F4F81F06051704792F0000F14BFA9
:1079500093F07F4F704730B54FF4607401F00045ED
:1079600021F0004120E700BF50EA010208BF704744
:1079700030B54FF000050AE050EA010208BF704739
:1079800030B511F0004502D5404261EB41014FF4A2
:10799000806404F132045FEA915C3FF4DCAE4FF0A6
:1079A00003025FEADC0C18BF03325FEADC0C18BF8D
:1079B000033202EBDC02C2F1200300FA03FC20FADE
:1079C00002F001FA03FE40EA0E0021FA02F114442B
:1079D000C1E600BF70B54FF0FF0C4CF4E06C1CEA40
:1079E00011541DBF1CEA135594EA0C0F95EA0C0FB5
:1079F00000F0DEF82C4481EA030621EA4C5123EA28
:107A00004C5350EA013518BF52EA033541F4801156
:107A100043F4801338D0A0FB02CE4FF00005E1FB09
:107A200002E506F00042E0FB03E54FF00006E1FB53
:107A300003569CF0000F18BF4EF0010EA4F1FF0496
:107A4000B6F5007F64F5407404D25FEA4E0E6D41D6
:107A500046EB060642EAC62141EA55514FEAC520E7
:107A600040EA5E504FEACE2EB4F1FD0C88BFBCF563
:107A7000E06F1ED8BEF1004F08BF5FEA500E50F114
:107A8000000041EB045170BD06F0004646EA0101DA
:107A900040EA020081EA0301B4EB5C04C2BFD4EB0C
:107AA0000C0541EA045170BD41F480114FF0000E05
:107AB000013C00F3AB8014F1360FDEBF002001F073
:107AC000004170BDC4F10004203C35DA0C341BDCED
:107AD00004F11404C4F1200500FA05F320FA04F0BF
:107AE00001FA05F240EA020001F0004221F00041F3
:107AF00010EBD37021FA04F642EB06015EEA430E66
:107B000008BF20EAD37070BDC4F10C04C4F1200595
:107B100000FA04F320FA05F001FA04F240EA020048
:107B200001F0004110EBD37041F100015EEA430E19
:107B300008BF20EAD37070BDC4F1200500FA05F239
:107B40004EEA020E20FA04F301FA05F243EA0203B8
:107B500021FA04F001F0004121FA04F220EA0200C7
:107B600000EBD3705EEA430E08BF20EAD37070BD0D
:107B700094F0000F0FD101F00046400041EB0101ED
:107B800011F4801F08BF013CF7D041EA060195F0CF
:107B9000000F18BF704703F00046520043EB030389
:107BA00013F4801F08BF013DF7D043EA0603704776
:107BB00094EA0C0F0CEA135518BF95EA0C0F0CD081
:107BC00050EA410618BF52EA4306D1D181EA0301C7
:107BD00001F000414FF0000070BD50EA410606BFC1
:107BE0001046194652EA430619D094EA0C0F02D106
:107BF00050EA013613D195EA0C0F05D152EA03364B
:107C00001CBF104619460AD181EA030101F0004168
:107C100041F0FE4141F470014FF0000070BD41F0B1
:107C2000FE4141F4780170BD70B54FF0FF0C4CF48B
:107C3000E06C1CEA11541DBF1CEA135594EA0C0FAA
:107C400095EA0C0F00F0A7F8A4EB050481EA030EF7
:107C500052EA03354FEA013100F088804FEA0333DE
:107C60004FF0805545EA131343EA12634FEA0222AC
:107C700045EA111545EA10654FEA00260EF000416D
:107C80009D4208BF964244F1FD0404F5407402D2BF
:107C90005B084FEA3202B61A65EB03055B084FEA50
:107CA00032024FF480104FF4002CB6EB020E75EB4D
:107CB000030E22BFB61A754640EA0C005B084FEA75
:107CC0003202B6EB020E75EB030E22BFB61A7546F2
:107CD00040EA5C005B084FEA3202B6EB020E75EB3D
:107CE000030E22BFB61A754640EA9C005B084FEAB5
:107CF0003202B6EB020E75EB030E22BFB61A7546C2
:107D000040EADC0055EA060E18D04FEA051545EAB0
:107D100016754FEA06164FEAC30343EA52734FEA59
:107D2000C2025FEA1C1CC0D111F4801F0BD141EAD2
:107D300000014FF000004FF0004CB6E711F4801F37
:107D400004BF01430020B4F1FD0C88BFBCF5E06F17
:107D50003FF6AFAEB5EB030C04BFB6EB020C5FEA27
:107D6000500C50F1000041EB045170BD0EF0004E7C
:107D70004EEA113114EB5C04C2BFD4EB0C0541EAAE
:107D8000045170BD41F480114FF0000E013C90E6AB
:107D900045EA060E8DE60CEA135594EA0C0F08BF6F
:107DA00095EA0C0F3FF43BAF94EA0C0F0AD150EA6E
:107DB00001347FF434AF95EA0C0F7FF425AF104601
:107DC00019462CE795EA0C0F06D152EA03353FF429
:107DD000FDAE1046194622E750EA410618BF52EAA6
:107DE00043067FF4C5AE50EA41047FF40DAF52EA7A
:107DF00043057FF4EBAE12E74FF0FF3C06E000BF17
:107E00004FF0010C02E000BF4FF0010C4DF804CD23
:107E10004FEA410C7FEA6C5C4FEA430C18BF7FEAE3
:107E20006C5C1BD001B050EA410C0CBF52EA430C11
:107E300091EA030F02BF90EA020F0020704710F191
:107E4000000F91EA030F58BF994208BF90422CBF20
:107E5000D8176FEAE37040F0010070474FEA410C19
:107E60007FEA6C5C02D150EA013C07D14FEA430C37
:107E70007FEA6C5CD6D152EA033CD3D05DF8040BA8
:107E8000704700BF8446104662468C4619466346DA
:107E900000E000BF01B5FFF7B7FF002848BF10F1B1
:107EA000000F01BD4DF808EDFFF7F4FF0CBF0120F6
:107EB00000205DF808FB00BF4DF808EDFFF7EAFF72
:107EC00034BF012000205DF808FB00BF4DF808ED2D
:107ED000FFF7E0FF94BF012000205DF808FB00BF22
:107EE0004DF808EDFFF7CEFF94BF012000205DF8AC
:107EF00008FB00BF4DF808EDFFF7C4FF34BF0120B9
:107F000000205DF808FB00BF4FEA410212F50012A5
:107F100015D211D56FF47873B3EB625212D94FEAD0
:107F2000C12343F0004343EA505311F0004F23FABA
:107F300002F018BF404270474FF00000704750EA0F
:107F4000013005D111F0004008BF6FF000407047CC
:107F50004FF00000704700BF4FEA4102B2F1E0432A
:107F600024BFB3F5001CDCF1FE5C0DD901F0004C20
:107F70004FEAC0024CEA5070B2F1004F40EB830070
:107F800008BF20F00100704711F0804F21D113F19C
:107F90003872BCBF01F00040704741F480114FEAD5
:107FA0005252C2F11802C2F1200C10FA0CF320FA5E
:107FB00002F018BF40F001004FEAC1234FEAD3237B
:107FC00003FA0CFC40EA0C0023FA02F34FEA4303E5
:107FD000CCE77FEA625307D150EA01331EBF4FF06E
:107FE000FE4040F44000704701F0004040F0FE4089
:107FF00040F40000704700BF704700BFFFFFFFFF65
:108000004A1E08BF7047C0F02481884240F21681A2
:10801000114200F01781B0FA80F3B1FA81F2A2EBBD
:108020000303C3F11F0304A202EB03134FF000028A
:108030009F4600BFAFF30080B0EBC17F00BF42EBB3
:10804000020228BFA0EBC170B0EB817F00BF42EB02
:10805000020228BFA0EB8170B0EB417F00BF42EB72
:10806000020228BFA0EB4170B0EB017F00BF42EBE2
:10807000020228BFA0EB0170B0EBC16F00BF42EB62
:10808000020228BFA0EBC160B0EB816F00BF42EBE2
:10809000020228BFA0EB8160B0EB416F00BF42EB52
:1080A000020228BFA0EB4160B0EB016F00BF42EBC2
:1080B000020228BFA0EB0160B0EBC15F00BF42EB42
:1080C000020228BFA0EBC150B0EB815F00BF42EBC2
:1080D000020228BFA0EB8150B0EB415F00BF42EB32
:1080E000020228BFA0EB4150B0EB015F00BF42EBA2
:1080F000020228BFA0EB0150B0EBC14F00BF42EB22
:10810000020228BFA0EBC140B0EB814F00BF42EBA1
:10811000020228BFA0EB8140B0EB414F00BF42EB11
:10812000020228BFA0EB4140B0EB014F00BF42EB81
:10813000020228BFA0EB0140B0EBC13F00BF42EB01
:10814000020228BFA0EBC130B0EB813F00BF42EB81
:10815000020228BFA0EB8130B0EB413F00BF42EBF1
:10816000020228BFA0EB4130B0EB013F00BF42EB61
:10817000020228BFA0EB0130B0EBC12F00BF42EBE1
:10818000020228BFA0EBC120B0EB812F00BF42EB61
:10819000020228BFA0EB8120B0EB412F00BF42EBD1
:1081A000020228BFA0EB4120B0EB012F00BF42EB41
:1081B000020228BFA0EB0120B0EBC11F00BF42EBC1
:1081C000020228BFA0EBC110B0EB811F00BF42EB41
:1081D000020228BFA0EB8110B0EB411F00BF42EBB1
:1081E000020228BFA0EB4110B0EB011F00BF42EB21
:1081F000020228BFA0EB0110B0EBC10F00BF42EBA1
:10820000020228BFA0EBC100B0EB810F00BF42EB20
:10821000020228BFA0EB8100B0EB410F00BF42EB90
:10822000020228BFA0EB4100B0EB010F00BF42EB00
:10823000020228BFA0EB0100104670470CBF0120CE
:1082400000207047B1FA81F2C2F11F0220FA02F059
:10825000704708B14FF0FF30FFF7CEBE0029F8D0CD
:108260002DE90340FFF7CCFEBDE8064002FB00F31A
:10827000A1EB0301704700BF03460846194600F012
:1082800009B800BF00210A2201F0D2B900220A2356
:1082900001F02CB930B405460C461346022029469D
:1082A000224630BC01F0D2B949F22003C1F6FF7377
:1082B0001868704770B54AF210364AF21035C0F2AD
:1082C0000006C0F20005761BB61007D0043D00245E
:1082D00055F8043F01349847A642F9D14AF24C368A
:1082E0004AF21035C0F20006C0F20005761B02F01B
:1082F00009F8B61008D0043D002455F8043F0134B5
:108300009847A642F9D170BD70BD00BF49F2200365
:108310000146C1F6FF73186800F008B849F220035F
:108320000146C1F6FF73186801F052BA2DE9F04F0B
:1083300001F10B04162C83B0074630D924F0070452
:10834000E30F8C422CBF194643F0010100292FD1C5
:10835000384600F06FFCB4F5FC7F2ED24FEAD40C07
:1083600049F21416C1F6FF7606EBCC02D3689342AD
:1083700000F01182596803F10808DA68384621F0E4
:10838000030499681B195C68CA6044F00104916099
:108390005C6000F051FC404603B0BDE8F08F002364
:1083A00010248C422CBF194643F001010029CFD084
:1083B0000C234FF000083B60EDE75FEA542C04BF4C
:1083C0004FEAD40C4FEA4C0540F08F8049F2141666
:1083D000C1F6FF7606EB8505EB689D4206D10DE000
:1083E000002A80F25581DB689D4207D0596821F050
:1083F00003010A1B0F2AF3DD0CF1FF3C0CF1010C09
:1084000049F214123369C1F6FF7202F1080E734586
:1084100008BFD2F8049022D0586820F00300011B56
:108420000F2900F384810029C2F814E0C2F810E09B
:1084300066DAB0F5007F80F04E81C1084FF0010888
:1084400002EBC100891008FA01F851688568D8600C
:1084500048EA0109C2F804909D60EB608360012244
:108460004FEAAC0302FA03F34B4554D819EA030F61
:108470000DD193402CF0030C19EA030F0CF1040CFE
:1084800005D15B000CF1040C19EA030FF9D006EBDF
:10849000CC09E0464846C268904207D15BE100291A
:1084A00080F28381D268904200F05581556825F0B2
:1084B0000305291B0F29F2DD90461319D56844F0F6
:1084C000010058F8084F41F0010C50603846C3F8DD
:1084D00004C0E560AC6073613361C3F80CE0C3F8BD
:1084E00008E0595000F0A8FB55E7BCF1040F00F27A
:1084F000DE804FEA941C0CF1380C4FEA4C0565E71E
:108500001A1803F108083846536843F00103536012
:1085100000F092FB3FE7B5686B6823F0030A54450F
:1085200004D8C4EB0A030F2B00F3A48044F274694F
:10853000D6F80814C2F2000905EB0A020131D9F895
:108540000030234408BF03F1100B06D003F580531D
:108550000F3323F47F6323F00F0B38465946019203
:1085600000F05CFD019A411C804600F06881824267
:1085700000F23181D9F8043042455B44C9F8043037
:1085800000F06681D6F8081449F21410C1F6FF70A5
:10859000013117BFC2EB0802C0F808849B18C9F864
:1085A000043018F0070338461FBFC3F10802C3F5B3
:1085B0008053904403F1080208EB0B0308BF4FF40B
:1085C00080521B051B0DC3EB020B594600F026FD24
:1085D000431C00F04981C8EB0001594441F00101FE
:1085E000D9F80430B54244F27462C6F808805B449E
:1085F000C2F20002C8F80410C9F8043018D0BAF169
:108600000F0F40F20B81AAF10C00696820F00700FF
:108610004FF0050C05EB000E0F2801F0010140EAB8
:1086200001016960CEF804C0CEF808C000F22081D4
:1086300044F27462D9F82C10C2F20002B5688B4281
:10864000D9F8301088BFD36244F27462C2F20002DB
:108650008B4288BF13636A6822F003029442C4EB22
:10866000020301D80F2B05DC38464FF0000800F05C
:10867000E3FA90E62A1943F0010344F00104384676
:108680006C6005F108085360B26000F0D5FA82E62C
:108690005918DA689C6838464D6803F1080845F0B7
:1086A0000105E26094604D6000F0C6FA73E6BCF12B
:1086B000140F9CBF0CF15B0C4FEA4C057FF686AEA5
:1086C000BCF1540F00F293804FEA143C0CF16E0C95
:1086D0004FEA4C057AE6420A042A75D9142A9CBF4F
:1086E00002F15B094FEA490508D9542A00F2C98012
:1086F0004FEA103909F16E094FEA490506EB850585
:1087000049F21418C1F6FF78AA68AA4279D05168D4
:1087100021F00301884202D292689542F7D1D068D5
:10872000D6F80490D8609A60D360836097E61D19EC
:1087300041F00106556144F00104156138465C6062
:1087400003F10808C5F80CE0C5F808E06E60695050
:1087500000F072FA1FE608F10108083018F0030F64
:108760007FF499AE4A461CF0030FA2F108010CF108
:10877000FF3C00F09E8012688A42F4D072685B0071
:1087800093423FF6C8AE002B3FF4C5AE1A4200F04C
:108790009580C4467BE603F108025B699A4208BFF4
:1087A0000CF1020C3FF42CAEE4E590465519D36869
:1087B000384658F8082F6968D36041F001019A6083
:1087C000696000F039FAE6E54FEA901909F13809D5
:1087D0004FEA490592E7B54249F21413C1F6FF7317
:1087E0003FF4C8AE9D686A6822F0030236E7BCF524
:1087F000AA7F19D84FEAD43C0CF1770C4FEA4C050C
:10880000E4E50125D8F804104FEAA909104605FA55
:1088100009F545EA0109C8F8049083E701234546B4
:10882000C8F80430002219E740F254539C450BD895
:108830004FEA944C0CF17C0C4FEA4C05C6E5B56848
:108840006A6822F0030209E7FC254FF07E0CBDE5C3
:108850001105090D00297FF495AEB2680BEB0A01F2
:1088600041F001015160E3E601214FF0000BB7E652
:10887000384605F10801019200F0AAFF019A5368F9
:10888000D6E6B2F5AA7F06D84FEAD03909F17709C2
:108890004FEA490532E740F25451FC258A424FF035
:1088A0007E099EBF4FEA904909F17C094FEA4905CC
:1088B00024E7726822EA0302726060E75B0008F155
:1088C000040863E7032A70B422D941EA00039B0736
:1088D00013D00578013A0C780023A54206D01BE09E
:1088E00010F8015F11F8014FA54215D1934203F131
:1088F0000103F5D1002070BC70470C4603460431DB
:1089000004301E682568AE4208D1043A032AF4D820
:10891000002ADED11046EEE7281BECE72146184678
:10892000002AD6D1F6E700BF032A2DE9F00F09D8B7
:108930002AB10023CC5CC45401339342FAD1BDE880
:10894000F00F7047830702440ED0441C4D1C15F8ED
:10895000017C04F00306234601342946013504F85E
:10896000027C002EF3D100E0034611F003046DD029
:10897000D71A0D1B032F2E6819DDC4F1040C4FEA22
:10898000C4081C1D4FEACC0C55F8047FC4EB020947
:10899000234604310434B9F1030F26FA08FA07FA22
:1089A0000CFB3E464BEA0A0744F8087CECDC9A4292
:1089B000C5D901330131013211F8014C01330131C4
:1089C000934203F8024CF7D1B9E70C6840334031C9
:1089D00043F8404C51F83C4C43F83C4C51F8384C6F
:1089E00043F8384C51F8344C43F8344C51F8304C7F
:1089F00043F8304C51F82C4C43F82C4C51F8284C8F
:108A000043F8284C51F8244C43F8244C51F8204C9E
:108A100043F8204C51F81C4C43F81C4C51F8184CAE
:108A200043F8184C51F8144C43F8144C51F8104CBE
:108A300043F8104C51F80C4C43F80C4C51F8084CCE
:108A400043F8084C51F8044C43F8044CD41A3F2C1A
:108A5000BBDC11E00C681033103143F8104C51F8B6
:108A60000C4C43F80C4C51F8084C43F8084C51F8A6
:108A7000044C43F8044CD41A0F2CEBDC032C96DD89
:108A80001C1D0D1D55F8047C161B23462946043475
:108A90000435032E44F8087CF4DC88E78842F0B4FF
:108AA00011D98C18A0420ED28518531E4AB1214606
:108AB0002A4611F8014D013BB3F1FF3F02F8014D89
:108AC000F7D1F0BC70470F2A47D941EA00039B0752
:108AD00045D10C4603461546266810331034103D28
:108AE0000F2D43F8106C54F80C6C43F80C6C54F8D0
:108AF000086C43F8086C54F8046C43F8046CEBD829
:108B0000A2F1100502F00F0425F00F051035032C1B
:108B100000EB0503294424D9A4F1040C1D460C469E
:108B20004FEA9C0C01EB8C07043754F8046BBC42F1
:108B300045F8046BF9D10CF1010402F00302A40022
:108B400009191B19002ABCD001399A1811F8014FD4
:108B500003F8014B9342F9D1B3E70346F2E703462A
:108B6000F2E72246EEE700BF032AC9B270B408D884
:108B70002AB10346121803F8011B9342FBD170BCC3
:108B800070478307024409D0441C04F003052346C0
:108B900004F8011C0134002DF7D100E00346D51A7A
:108BA00001EB01243F2D04EB04442CDD1C60403319
:108BB000D51A43F83C4C3F2D43F8384C43F8344C1D
:108BC00043F8304C43F82C4C43F8284C43F8244CE1
:108BD00043F8204C43F81C4C43F8184C43F8144C11
:108BE00043F8104C43F80C4C43F8084C43F8044C41
:108BF000DCDC08E01C601033D51A43F80C4C43F859
:108C0000084C43F8044C0F2DF4DC032D08DD1D1D2A
:108C1000561B45F8044C032E2B4605F10405F7DCE2
:108C20009A42ACD90133013203F8011C013393425B
:108C3000FAD1A4E7704700BF704700BF49F2200394
:108C40000A46C1F6FF730146186800F001B800BF7C
:108C50002DE9F04F0C4683B081461746002900F0FD
:108C60001C8107F10B05FFF7E5FF54F8042C162DC6
:108C7000A4F1080A22F0030675D8102100230D463E
:108C8000BD4238BF43F00103002B40F00C818E42FF
:108C90006EDA49F2141B0AEB0600C1F6FF7BDBF823
:108CA00008E0864500F00481D0F804C02CF00108EB
:108CB0008044D8F8048018F0010F1CBF9C46604621
:108CC0006FD0D30700F1C38054F8083CC3EB0A030C
:108CD0005A6822F003029219019200286CD0704564
:108CE00000F037810CEB0208884565DBC1681F4640
:108CF0008068321F242A8860C16057F8080FD9683D
:108D0000C160886000F27881132A9CBF39462046F2
:108D10001FD921681B2A98BF04F108009960616877
:108D2000D96098BF03F1100113D9A168242A14BF98
:108D300004F1100004F118001961E168596111BFD4
:108D400003F11801226903F120019A6104BF6269ED
:108D5000DA6102683C460A609A4642684A60826864
:108D60008A605A6805E025F007052946EB0F87E77A
:108D7000B046C5EB08030F2B55D80AEB080302F0E9
:108D8000010242EA0802CAF804205A6842F00102CD
:108D90005A6048462746FFF74FFF384603B0BDE804
:108DA000F08F2CF0030C0CEB0608884589DBC368B8
:108DB0008168CB609960DCE7019A8A4247DB1F46F5
:108DC000D968321F57F8080F242AC160886000F262
:108DD000B180132A9CBF394620461FD921681B2A1F
:108DE00098BF04F1080099606168D96098BF03F1E9
:108DF000100113D9A168242A14BF04F1100004F152
:108E000018001961E168596111BF03F11801226965
:108E100003F120019A6104BF6269DA6102683C468D
:108E2000DDF8048097E70AEB050102F00102CE1895
:108E3000154343F00103CAF804504B604846736879
:108E4000083143F00103736000F0C2FCA1E739462A
:108E50004846FFF76BFA0746D8B154F8042CA0F146
:108E6000080122F001035344994200F0BF80321FF1
:108E7000242A6AD8132A9CBF0346224639D811688F
:108E800019605168596092689A604846214600F01E
:108E90009FFC4846FFF7D0FE7FE7114603B0BDE8D0
:108EA000F04FFFF743BA0C230027C9F8003074E7EE
:108EB000DEF8043005F1100023F0030C0CEB060380
:108EC0008342B8BF7046FFF6FCAE0AEB05025B1B9F
:108ED00043F0010348465360274654F8043CCBF85E
:108EE000082003F001031D4344F8045CFFF7A4FECF
:108EF00053E723681B2A98BF04F1080203606368E4
:108F0000436098BF00F10803B9D9A368242A14BFAD
:108F100004F1100204F118028360E368C36011BF1A
:108F200000F11003216900F11803016104BF6169B8
:108F30004161A4E7214638460093FFF7AFFD9DE865
:108F400008013C469A465A6813E72146FFF7A6FDFA
:108F50009BE7019805F110020CEB00089045FFF625
:108F60002BAF1F46D968321F57F8080F242AC1605B
:108F700088604BD8132A9CBF3A4621461FD92168E6
:108F80001B2A98BF03F1100299606168D96098BFED
:108F900004F1080113D9A168242A14BF03F11802AF
:108FA00003F120021961E168596111BF04F1100158
:108FB000206904F11801986104BF6069D8610868EC
:108FC000106048685060896891605A19C5EB0801C3
:108FD00041F00101484651605968CBF8082001F082
:108FE00001010D435D60FFF727FED6E650F8043C13
:108FF00023F00308B044BCE6214638460093FFF74F
:109000004DFD009B3C469A465A68B2E638462146DA
:109010000093FFF743FD009BD7E700BF38B544F24C
:10902000B864C2F200040546084600232360FAF73C
:1090300041FE431C00D038BD2368002BFBD02B60C1
:1090400038BD00BFC9B2F0B400294BD083070FD0A0
:109050000378002B73D0994242D0431C05E013F8EB
:10906000012B002A3BD091423AD09A071846F6D1FC
:10907000036841EA0127A3F1013247EA074722EAE0
:10908000030212F0803F1CD17B40A3F1013222EA9F
:10909000030313F0803F14D1021D02E014F0803F5F
:1090A0000FD1104652F8043BA3F1013687EA0304BE
:1090B00026EA0303A4F1013513F0803F25EA0404F6
:1090C000ECD00378002B3AD0994209D0431C01E040
:1090D000914205D0184613F8012B002AF8D110460A
:1090E000F0BC704781070DD00378002BF8D0431CEB
:1090F00002E00278002AF3D013F0030F184603F1C0
:109100000103F6D10368A3F1013222EA030313F04D
:10911000803F0AD1021D104652F8041BA1F1013410
:1091200024EA010111F0803FF5D00378002BD7D05D
:10913000431C184601330278002AFAD1D0E71846BA
:10914000CEE700BF80EA010212F0030F40F03A8040
:1091500010F0030220F0030021F0030150F804CBCB
:1091600008BF51F8043B0DD082F003024FEAC2025F
:109170006FF07F4323FA02F251F8043B4CEA020CF1
:1091800043EA0203ACF101329C4501BF22EA0C0222
:1091900012F0803F50F804CB51F8043BF2D04FEA74
:1091A0000C604FEA1C2C012828BFB0EB036F08BFEE
:1091B0001B0AF4D003F0FF034FEA1060A0EB03009A
:1091C000704700BF10F0030F0AD010F8012B11F800
:1091D000013B012A28BF9A42F4D0A2EB030070475A
:1091E0004DF8045D4DF8044D4FF0010242EA0222B1
:1091F00042EA024201F0030C21F0030150F8044B53
:1092000051F8045BBCF1020F26D04BD824F07F4C00
:10921000BCEB152FA4EB020323EA04030DD113EAE0
:10922000C21308BF51F8045B0AD18CEA040CBCEBF2
:10923000056F0CD150F8044BE8E74FEA15255CE0C8
:1092400033F07F4352D10D784FEA146C55E04FEA6A
:10925000146C05F0FF0550E04FEA044CA4EB020348
:109260004FEA1C4C23EA0403BCEB154F17D113EA59
:10927000C21308BF51F8045B07D18CEA040CBCEBA5
:10928000054F08D150F8044BE6E71B042ED10D889A
:109290004FEA144C31E04FEA05454FEA144C4FEACF
:1092A00015452AE004F0FF0CBCEB156FA4EB02039C
:1092B00023EA04030DD113EAC21308BF51F8045B7B
:1092C0000AD18CEA040CBCEB052F0AD150F8044BF0
:1092D000E8E74FEA156510E014F0FF0F06D051F8EB
:1092E000045B4FEA142C25F07F4506E04FF00000A8
:1092F0005DF8044B5DF8045B70470CF0FF0205F06D
:10930000FF00012828BF904204BF4FEA1C2C2D0A01
:10931000F3D0A2EB00005DF8044B5DF8045B7047EE
:1093200080EA0102844612F0030F4FD111F0030FBF
:1093300032D14DF8044D11F0040F51F8043B0BD01D
:10934000A3F101329A4312F0803F04BF4CF8043B72
:1093500051F8043B16D100BF51F8044BA3F1013280
:109360009A4312F0803FA4F101320BD14CF8043B38
:10937000A24312F0803F04BF51F8043B4CF8044B69
:10938000EAD023460CF8013B13F0FF0F4FEA3323DA
:10939000F8D15DF8044B704711F0010F06D011F8B9
:1093A000012B0CF8012B002A08BF704711F0020FA7
:1093B000BFD031F8022B12F0FF0F16BF2CF8022B92
:1093C0008CF8002012F47F4FB3D1704711F8012BB5
:1093D0000CF8012B002AF9D1704700BF70B4002AA5
:1093E00045D041EA000313F0030329D1032A27D90A
:1093F00005680C68A54223D1141F3AD0A5F10132AB
:1094000022EA050515F0803F0DD03AE05B686A68F6
:10941000A3F10135934225EA03052ED1043C28D05F
:1094200015F0803F27D10D46034604310430032C4C
:10943000ECD8661E2CB91C792A79A01A70BC70472A
:10944000561E04780A789442F7D1C6B18CB1013621
:109450008B1C891904E08B4203F101030BD044B14A
:1094600013F8012C10F8014F9442F4D0E5E71046B0
:10947000E4E72046E2E70020E0E7661EE1E7304649
:10948000DCE71846DAE700BF41EA000313F0030FF8
:10949000034670B425D0AAB10C78013A03F8014B09
:1094A0004CB11C4672B111F8015F013A04F8015B3E
:1094B0002346002DF6D12AB19A18002103F8011B8A
:1094C0009342FBD170BC70470E4651F8044BA4F197
:1094D000013525EA040515F0803F05D1043A43F82B
:1094E000044B032AF0D8D6E73146D4E72DE9F04FF4
:1094F00049F22454C1F6FF7485B099460B46D4F85E
:109500000080029103901C4614F8015B08EB0501F2
:109510002346497801F00801C9B20029F3D12D2D65
:109520007BD02B2D05BF24460B460B4614F8015B60
:1095300039F0100112D1D9F1010038BF0020302DCF
:1095400004D058B14FF00A09CB4608E0217801F069
:10955000DF01582965D008B14FF00809CB46002B30
:1095600059460CBF6FF000464FF000468DE80C00E6
:1095700030460027FEF772FE30468A465946FEF70F
:109580003FFDBC469DE80C0016E0303DA94525DDB9
:10959000844594BF0021012151EAD77729D155454F
:1095A000D4BF00210121844518BF002109BB0BFB5A
:1095B0000C5C012714F8015B08EB0501497801F008
:1095C0000406F6B2002EE0D111F0030106D0012905
:1095D00014BF572137216D1AA945D9DC791C0BD04E
:1095E000C3B9604612B197B9029B136005B0BDE8DC
:1095F000F08F4FF0FF37DDE70399002B0CBF6FF0C2
:1096000000404FF0004022230B60002AEED0013CC6
:109610000294E9E7CCF1000CE3E714F8015B0123C5
:1096200086E74FF010096578CB46023497E700BF14
:1096300030B449F22004C1F6FF740D4613460146CA
:109640002A46206830BCFFF751BF00BF2DE9F0412A
:109650004AF29814C0F2000484B007462568AC6C46
:10966000002C42D066681F2E1ADD48F20D34C0F27D
:10967000000424B94FF0FF3004B0BDE8F0818C2025
:10968000039102920193FEF741FE0399029A019B16
:1096900004460028EED0A86C002684E84100AC64A3
:1096A000DFB1D4F8886026B3D6F800816568012060
:1096B000022F05F1200C00FA05F046F8252048EAB3
:1096C000000246F82C3008BFD6F80431C6F8002155
:1096D00004BF1843C6F8040100E06568AB1C002015
:1096E0000135656044F82310C6E705F14C04AC640D
:1096F000B8E748F20D30C0F200000028BAD04FF4AD
:109700008470039102920193FEF700FE0399029A7E
:10971000019B06460028ADD00020C6F80001C6F81F
:1097200004018046C4F88860C0E700BFF8B549F27C
:109730001414C1F6FF740F460546FFF77BFAA368C1
:109740005E6826F0030606F6EF73DF1B3F0B013F52
:109750003F03B7F5805F07DB00212846FFF75EFC7B
:10976000A3689B19984204D02846FFF765FA0020A9
:10977000F8BD79422846FFF751FC013010D044F281
:109780007863A168C2F20003F61B284646F0010682
:109790001A684E60D71B1F60FFF74EFA0120F8BD14
:1097A00000212846FFF73AFCA368C21A0F2ADBDD26
:1097B00049F21C5444F27861C1F6FF74C2F2000110
:1097C00042F001025A602368C01A0860CCE700BF6B
:1097D0002DE9F0410E46804600295CD0FFF72AFAB9
:1097E00049F2141556F8041CC1F6FF75A6F10804D9
:1097F00021F00103AF68E2189742506820F003009F
:1098000067D011F00101506035D00021161876683C
:1098100016F0010F06D11B18906800294DD0D268B0
:10982000C260906043F00102E3506260F1B9B3F5A9
:10983000007F32D35A0A042A6CD898093830410084
:1098400005EB810549F21411C1F6FF71AA68AA421D
:109850006BD0516821F003018B4202D2926895428D
:10986000F7D1D368E360A260D4609C604046BDE855
:10987000F041FFF7E1B956F8086C05F1080CA41B9C
:109880009B19A668664543D0D4F80CC0C6F80CC036
:10989000CCF80860BAE7BDE8F081DB080121686810
:1098A00005EBC3029B1001FA03F3E26091681843D1
:1098B0006860A160CC609460D8E7294EB042AED118
:1098C0006C6143F001022C61E060A0606260E350D3
:1098D000CCE7C018CB0707D456F8083CE41AC018E8
:1098E000A268E368D3609A6049F2205240F0010315
:1098F000C1F6FF726360AC6013689842B6D344F25D
:1099000074634046C2F200031968FFF70FFFADE72A
:1099100001217BE702F15B004100142A90D9542A0F
:109920000CD8180B6E3041008AE701264D68801074
:10993000134606FA00F005434D6093E7B2F5AA7F9F
:1099400003D8D80B773041007AE740F254518A426D
:1099500003D8980C7C30410072E7FC217E206FE731
:109960001C91FF1FFFFFFFFF000000000000000030
:10997000C53C0000000000005F0053504F544C00F5
:109980005452415348002F00706F73004368616E5A
:109990006E656C20706F74207261773D00204368A3
:1099A000616E6E656C204356207261773D002043E6
:1099B0006F6D62696E6564207261773D0020636F30
:1099C0006E73747261696E65643D002066696C65D2
:1099D00020636F756E743D00206D61707065643D2D
:1099E000002A46696C6520456E6465642A002A2A4F
:1099F0002A2A2A4558504C4F44452A2A2A2A0049E7
:109A00006E206368616E676520626C6F636B2C20EB
:109A10004F6666736574203D200020506C61796844
:109A2000656164203D00205265736574203D00200F
:109A30004348414E4E454C203D00206661696C65AF
:109A4000643D002A46696C652053746172746564D4
:109A50003A00496E206D61696E206C6F6F702C202A
:109A60004F66667365743D200020706C617954699F
:109A70006D653D007C0042616E6B3A002043686179
:109A80006E6E656C3A002046696C653A0042616E04
:109A90006B3A20002046696C657320666F756E64B2
:109AA00000292000207C20005374617274696E6765
:109AB0002075702E2E2E00536574206D656D6F72AB
:109AC000792E2E2E005344206361726420736574D6
:109AD00074696E67202E2E2E00556E61626C6520B3
:109AE000746F2061636365737320746865205344E9
:109AF000206361726400534420636172642069735F
:109B0000204F4B202E2E2E004F70656E20526F6F0F
:109B100074202E2E2E005363616E2064697265637B
:109B2000746F72696573202E2E2E005241570030DB
:109B300000FF0000010004000B0013001E002C00B9
:109B40003C004E0063007B009500B100D000F100A6
:109B500014013A0163018E01BB01EA011D025102A9
:109B60008802C102FC023A037B03BD0302044904DC
:109B70009304DF042D057D05D00524067C06D5065B
:109B800030078E07EE075008B4081A098309ED095B
:109B90005A0AC90A390BAC0B210C980C100D8B0D0D
:109BA000080E860E070F890F0D1093101B11A511BB
:109BB0003112BE124D13DE13701404159A153216AD
:109BC000CB16651701189F183E19DF19811A251B3E
:109BD000CA1B711C181DC21D6C1E181FC51F7320C7
:109BE0002321D42186223923ED23A22458250F26B0
:109BF000C82681273B28F628B2296F2A2D2BEC2B6B
:109C0000AB2C6B2D2C2EED2EAF2F72303531F93160
:109C1000BD32823348340E35D4359B36623729380D
:109C2000F138B939813A493B123CDB3CA43D6D3EE9
:109C3000363FFF3FC84091415A422343EB43B4446F
:109C40007C4545460C47D4479C486349294AF04A1D
:109C5000B64B7B4C404D044EC84E8C4F4E5010516D
:109C6000D251935253531254D0548E554B560757DA
:109C7000C2577C583659EE59A55A5C5B115CC55CDD
:109C8000785D2A5EDB5E8A5F3960E66091613C62E6
:109C9000E5628D633364D9647C651E66BF665F6769
:109CA000FC6798683369CC69646AF96A8E6B206CCA
:109CB000B16C406DCD6D596EE26E6A6FF06F75706C
:109CC000F7707871F6717372EE726673DD735274A9
:109CD000C5743675A47511767B76E4764A77AE77CF
:109CE00010787078CE7829798379DA792F7A817A29
:109CF000D27A207B6C7BB57BFC7B417C847CC47CF2
:109D0000027D3E7D777DAE7DE27D147E447E717E58
:109D10009C7EC47EEA7E0E7F2F7F4E7F6A7F847F8B
:109D20009B7FB07FC37FD37FE17FEC7FF47FFB7F9E
:109D3000FE7FFF7FFFFFFFFF00000000000000002C
:109D400011160000000000000000000000000000EC
:109D5000511600000000000000000000000000009C
:109D60006D1800000000000000000000000000006E
:109D70005D1A0000000000006E203D004E4F3A20AA
:109D8000756E61626C6520746F206F70656E206601
:109D9000696C65005945533A2061626C6520746FA7
:109DA000206F70656E2066696C6500FFFFFFFFFF26
:109DB0000000000000000000491C0000E51C00003D
:109DC000851C0000991C0000C11C0000811C0000C3
:109DD0000200030004000500060008000A000C0051
:109DE0001000140018002000280038004000600017
:109DF0008000C00000018001000280020003FFFF1C
:109E000000000080000001800000000000000280CF
:109E1000000001000110000000000200011001001C
:109E200003200000010002000320010004300000B4
:109E3000032002000320030005400000054001004C
:109E40000650000006500100076000000760010096
:109E5000087000000760020008700100FFFFFFFFAC
:109E60000000000000000000C91F0000E71F000004
:109E7000212100002B2000003D200000DD1F0000FC
:109E80007C3C3E5E2B3D3F2F5B5D3B2C2A225C00E1
:109E90000000000000000000D134000089500000E4
:109EA000050E08090D0C06070F04001303931A9200
:109EB00017C585848687C4FF6FF07F03037003781E
:109EC00013F0800FFBD070474008FE4340A00440D1
:109ED0004408FE4344A004400018FE4300C0044070
:109EE0003000FE43309004403400FE433490044080
:109EF0001C18FE431CC004401018FE4310C0044050
:109F00000818FE4308C004400C18FE430CC004406F
:109F10000C10FE430CB004401010FE4310B004407F
:109F20001810FE4318B004401C10FE431CB004403F
:109F30001410FE4314B004400418FE4304C004404F
:109F40000010FE4300B004400008FE4300A004409F
:109F50000408FE4304A004400C08FE430CA0044087
:109F60000808FE4308A004401418FE4314C004402F
:109F70001818FE4318C004400410FE4304B0044007
:109F80000810FE4308B004401400FE43149004403F
:109F90004C08FE434CA004400420FE4304D004407F
:109FA0002410FE4324B004402010FE4320B004409F
:109FB0002810FE4328B004402C10FE432CB004406F
:109FC0000020FE4300D004404808FE4348A004405F
:109FD0001000FE43109004400D0AFFFFFFFFFFFF3B
:109FE0000000000000000000935100008B510000B1
:109FF000A5510000A15100009D51000099510000A1
:10A000000015191500010000808FFF1F12000000CD
:10A0100000020000AA8FFF1F4300000000030000A1
:10A020000490FF1F0000000001030904928FFF1F2E
:10A030000000000002030904EE8FFF1F0000000073
:10A04000030309040890FF1F000000000000000047
:10A050000000000000000000000000000000000000
:10A0600031610000556100007961000071610000FC
:10A07000756100006D61000087610000996100005A
:10A08000836100007D61000069610000656100007E
:10A09000F5600000016100000D6100001961000021
:10A0A0003D6100002561000000000000000000008C
:10A0B00015620000396200005D6200005562000018
:10A0C00059620000516200006B6200007D62000076
:10A0D00067620000616200004D620000496200009A
:10A0E000D9610000E5610000F1610000FD61000040
:10A0F0002162000009620000000000000000000072
:10A10000F96200001D630000416300003963000034
:10A110003D630000356300004F6300006163000091
:10A120004B63000045630000316300002D630000B5
:10A13000BD620000C9620000D5620000E16200005B
:10A1400005630000ED620000706F7700FFFFFFFF06
:10A15000000000000000F03F000000000000F83F99
:10A16000000000000000000006D0CF43EBFD4C3E95
:10A1700000000000000000000000004003B8E23FC3
:10A1800000FFFFFFFFFFFFFF000000000000304363
:10A1900000000000000030C32490FF1F43000000B7
:10A1A00000202020202020202020282828282820A7
:10A1B000202020202020202020202020202020209F
:10A1C0002088101010101010101010101010101007
:10A1D00010040404040404040404041010101010F7
:10A1E00010104141414141410101010101010101C1
:10A1F0000101010101010101010101011010101013
:10A200001010424242424242020202020202020292
:10A2100002020202020202020202020210101010E6
:10A22000200000000000000000000000000000000E
:10A23000000000000000000000000000000000001E
:10A24000000000000000000000000000000000000E
:10A2500000000000000000000000000000000000FE
:10A2600000000000000000000000000000000000EE
:10A2700000000000000000000000000000000000DE
:10A2800000000000000000000000000000000000CE
:10A2900000000000000000000000000000000000BE
:10A2A00000000000000000000000000000000000AE
:10A2B000000000000000000000000000000000009E
:10A2C000000000000000000000000000000000008E
:10A2D000000000000000000000000000000000007E
:10A2E000000000000000000000000000000000006E
:10A2F000000000000000000000000000000000005E
:10A3000000000000F8B500BFF8BC08BC9E467047CE
:10A3100099040000311300006B150000B517000010
:10A32000CD170000151A00002D1A0000451A000074
:10A33000B51E0000112500006D2C0000AD5100007D
:0CA34000BD610000A16200008563000008
:10A34C00000000000100000005000000FA00000001
:10A35C00FFFFFFFF0A040000BC460020FFFFFFFFC9
:10A36C001201000202000040C01683040001010229
:10A37C00030118035400650065006E00730079003A
:10A38C006400750069006E006F0009024300020151
:10A39C0000C0320904000001020201000524001073
:10A3AC00010524010101042402060524060001070D
:10A3BC0005820310004009040100020A0000000796
:10A3CC00050302400000070584024000000016034C
:10A3DC0055005300420020005300650072006900D4
:10A3EC0061006C00040309040C0300000000000071
:10A3FC000000000000000000000000000000010050
:10A40C002490FF1F00000000E4A20000C4A2000082
:10A41C00A4A20000000000000000000000000000EA
:10A42C00000000009CA100000000000000000000E3
:10A43C000000000000000000000000000000000010
:10A44C000000000000000000000000000000000000
:10A45C0000000000000000000000000000000000F0
:10A46C0000000000000000000000000000000000E0
:10A47C0000000000000000000000000000000000D0
:10A48C0000000000000000000000000000000000C0
:10A49C0000000000000000000000000000000000B0
:10A4AC0000000000000000000000000000000000A0
:10A4BC000000000000000000000000000000000090
:10A4CC000000000000000000000000000000000080
:10A4DC000000000000000000000000000000000070
:10A4EC000000000000000000000000000000000060
:10A4FC000000000000000000000000001491FF1F8D
:10A50C001491FF1F1C91FF1F1C91FF1F2491FF1F13
:10A51C002491FF1F2C91FF1F2C91FF1F3491FF1FC3
:10A52C003491FF1F3C91FF1F3C91FF1F4491FF1F73
:10A53C004491FF1F4C91FF1F4C91FF1F5491FF1F23
:10A54C005491FF1F5C91FF1F5C91FF1F6491FF1FD3
:10A55C006491FF1F6C91FF1F6C91FF1F7491FF1F83
:10A56C007491FF1F7C91FF1F7C91FF1F8491FF1F33
:10A57C008491FF1F8C91FF1F8C91FF1F9491FF1FE3
:10A58C009491FF1F9C91FF1F9C91FF1FA491FF1F93
:10A59C00A491FF1FAC91FF1FAC91FF1FB491FF1F43
:10A5AC00B491FF1FBC91FF1FBC91FF1FC491FF1FF3
:10A5BC00C491FF1FCC91FF1FCC91FF1FD491FF1FA3
:10A5CC00D491FF1FDC91FF1FDC91FF1FE491FF1F53
:10A5DC00E491FF1FEC91FF1FEC91FF1FF491FF1F03
:10A5EC00F491FF1FFC91FF1FFC91FF1F0492FF1FB2
:10A5FC000492FF1F0C92FF1F0C92FF1F1492FF1F5F
:10A60C001492FF1F1C92FF1F1C92FF1F2492FF1F0E
:10A61C002492FF1F2C92FF1F2C92FF1F3492FF1FBE
:10A62C003492FF1F3C92FF1F3C92FF1F4492FF1F6E
:10A63C004492FF1F4C92FF1F4C92FF1F5492FF1F1E
:10A64C005492FF1F5C92FF1F5C92FF1F6492FF1FCE
:10A65C006492FF1F6C92FF1F6C92FF1F7492FF1F7E
:10A66C007492FF1F7C92FF1F7C92FF1F8492FF1F2E
:10A67C008492FF1F8C92FF1F8C92FF1F9492FF1FDE
:10A68C009492FF1F9C92FF1F9C92FF1FA492FF1F8E
:10A69C00A492FF1FAC92FF1FAC92FF1FB492FF1F3E
:10A6AC00B492FF1FBC92FF1FBC92FF1FC492FF1FEE
:10A6BC00C492FF1FCC92FF1FCC92FF1FD492FF1F9E
:10A6CC00D492FF1FDC92FF1FDC92FF1FE492FF1F4E
:10A6DC00E492FF1FEC92FF1FEC92FF1FF492FF1FFE
:10A6EC00F492FF1FFC92FF1FFC92FF1F0493FF1FAD
:10A6FC000493FF1F0C93FF1F0C93FF1F1493FF1F5A
:10A70C001493FF1F1C93FF1F1C93FF1F2493FF1F09
:10A71C002493FF1F2C93FF1F2C93FF1F3493FF1FB9
:10A72C003493FF1F3C93FF1F3C93FF1F4493FF1F69
:10A73C004493FF1F4C93FF1F4C93FF1F5493FF1F19
:10A74C005493FF1F5C93FF1F5C93FF1F6493FF1FC9
:10A75C006493FF1F6C93FF1F6C93FF1F7493FF1F79
:10A76C007493FF1F7C93FF1F7C93FF1F8493FF1F29
:10A77C008493FF1F8C93FF1F8C93FF1F9493FF1FD9
:10A78C009493FF1F9C93FF1F9C93FF1FA493FF1F89
:10A79C00A493FF1FAC93FF1FAC93FF1FB493FF1F39
:10A7AC00B493FF1FBC93FF1FBC93FF1FC493FF1FE9
:10A7BC00C493FF1FCC93FF1FCC93FF1FD493FF1F99
:10A7CC00D493FF1FDC93FF1FDC93FF1FE493FF1F49
:10A7DC00E493FF1FEC93FF1FEC93FF1FF493FF1FF9
:10A7EC00F493FF1FFC93FF1FFC93FF1F0494FF1FA8
:10A7FC000494FF1F0C94FF1F0C94FF1F1494FF1F55
:10A80C001494FF1F1C94FF1F1C94FF1F2494FF1F04
:10A81C002494FF1F2C94FF1F2C94FF1F3494FF1FB4
:10A82C003494FF1F3C94FF1F3C94FF1F4494FF1F64
:10A83C004494FF1F4C94FF1F4C94FF1F5494FF1F14
:10A84C005494FF1F5C94FF1F5C94FF1F6494FF1FC4
:10A85C006494FF1F6C94FF1F6C94FF1F7494FF1F74
:10A86C007494FF1F7C94FF1F7C94FF1F8494FF1F24
:10A87C008494FF1F8C94FF1F8C94FF1F9494FF1FD4
:10A88C009494FF1F9C94FF1F9C94FF1FA494FF1F84
:10A89C00A494FF1FAC94FF1FAC94FF1FB494FF1F34
:10A8AC00B494FF1FBC94FF1FBC94FF1FC494FF1FE4
:10A8BC00C494FF1FCC94FF1FCC94FF1FD494FF1F94
:10A8CC00D494FF1FDC94FF1FDC94FF1FE494FF1F44
:10A8DC00E494FF1FEC94FF1FEC94FF1FF494FF1FF4
:10A8EC00F494FF1FFC94FF1FFC94FF1F0495FF1FA3
:10A8FC000495FF1F0C95FF1F0C95FF1FFFFFFFFF1B
:08A90C0000000200A0A1000000
:00000001FF
